:020000041100E9
:10300000002373B52B4D2C4C28006361022601F080
:1030100067F94021FE2221742800284B009601F018
:10302000B1F9002836D1217CFF222800244B0096DC
:1030300001F0A8F900282DD1224BA2899A4226D16D
:10304000E389214A93420DD1204B6361204B2268D2
:10305000002A03D1002B01D043CB43C4280001F048
:103060007DF973BD1B4A934201D00023EFE71A4B51
:103070001A4A1B68934206D9C02304222800217CE7
:103080009B0001F0F5F9114B6361154BDFE700235D
:103090002374EAE7CC233821AC2228009B01217459
:1030A00001F0E6F90028F2D10E4B63610E4BE3818B
:1030B0000E4BCCE7AC42FF1F7862FF1F8462FF1FFC
:1030C0008662FF1F59590000830500000D41001161
:1030D000FCBC0011821500009C62FF1F87130000DA
:1030E00008BD0011C5410011AAAAFFFFF0BC0011E4
:1030F000F7B5164B0192C318021D002000938823D8
:103100005B05D3181B685C1C1AD09CB2402C18D8E5
:103110008D781E0CAC466746CD782D023D43AE42FD
:1031200006D1019800280ED110000C70240A4C70B2
:1031300003249BB20733A343D218009B9A42DED3E9
:10314000FEBD4432F9E71000FAE7C046FC0F00006C
:10315000802213B503000324019189B25201073183
:103160009B18A14304305A1A88235B05C3181B68B7
:10317000591C03D190429241104016BD99B240298A
:1031800007D80B000733A343C0189042ECD30020AC
:10319000F3E74430F9E7134B134A1B68126810B584
:1031A000FA24934201D81A00F824104BE4021B6859
:1031B0009A4210D813000E4A12689A420ED3013375
:1031C00007D1F823DB029C4203D10A49054808F0E5
:1031D000E3FA200010BDFC24E402ECE7FE24E40244
:1031E000F7E7C04600C0071100D0071100E0071143
:1031F00000F00711FFFFFF7FF0B59BB015000490B2
:103200000391402A00D9A0E006AB59801A80FFF74D
:10321000C2FF0400042816D9002206A9FFF768FFA0
:10322000052810D906AB1B88AB420CD1002D07D066
:10323000514B2A000499C01808F0BEFC002802D1A6
:1032400001201BB0F0BD06AB1D8020000699FFF7E2
:103250007FFF041E7BD1069B0793FFF79CFF802313
:103260005B01C618802307001B039E4201D3F8268A
:10327000F60288235B05F31801931B68013302D023
:10328000019808F011FB3D49019808F085FA3B1DB3
:103290000293331D05938822029B52059B181B68DD
:1032A00008935A1C3CD044219AB20091402A04D879
:1032B0000320D11D814389B2009103991B0C8B42DD
:1032C00024D0402A22D80122300008A9FFF710FF9D
:1032D000021E1BD1380008A9FFF70AFF04000428CA
:1032E00031D9009A059B9B1880225201B218934253
:1032F00040D288235B05C118009A09A808F0B4FBE6
:103300001D4B009A09A9F01808F0C6FB009A029B11
:103310009446634402931A4B029AFB189A42BAD31A
:1033200088235B05FC1821680198013908F034FAFC
:10333000200008F0B9FA039A07AB5A8030000799C9
:10334000FFF706FF0400002C03D1002079E70428D2
:10335000FBD988235B05E018069908F01DFA0323C2
:10336000EA1C9A4300D16BE7034B0499E01808F07C
:1033700093FB65E70424ECE704000011FFFFFF7FE7
:10338000F80F0000F7B505001400402A21D80027E7
:1033900001AE71803780FFF7FEFE042816D93A008F
:1033A0003100FFF7A5FE042810D93688BC420BD0A7
:1033B000BD4209D0221CB44200D9321C064B92B245
:1033C000C118280008F050FB30B2FEBDC04300B267
:1033D000FBE703204042F8E70400001137B5042260
:1033E00004000D0001A81649FFF7CCFF02000428D5
:1033F0000BD1019BA34208D3AB4204D0104901A8D2
:103400000195FFF7F9FE01203EBD0E4C2368200018
:10341000019308F049FA019920000139019108F05F
:10342000BBF980235B01E418074B9C42EED10422D8
:10343000034901A80195FFF7DFFE0020E4E7C0463D
:103440005555000000C007110000081130B589B0C3
:1034500008F04AFA10226946254808F075F9254B0C
:10346000009A9A420ED1019B029A0F2B33D8002169
:1034700001240698013B08D2002900D00292029B49
:10348000013331D10023029325E0551CF2D1020013
:103490002100EFE710341022200004A908F054F9AD
:1034A000029B013301D1069B0293882304995B059B
:1034B000C918059B06981A03120B049105928142C4
:1034C00003D02B4201D108F0CFFA019B013B0193BD
:1034D000019B002BDED1029B002B03D004930498A8
:1034E0004168084709B030BDE025014C2D03EFE7E6
:1034F00000000111504859368022F8B5964C974B80
:10350000D200002120001C6008F006FB2300944A32
:1035100088331A60934B1A786A23002A00D011333B
:10352000E3620A232365904B37221B780820A363AC
:103530008E4B2118E361102323628D4B3B25636181
:10354000C823DB00A36123008C331A602823013ACF
:10355000E26320646364CA67043A211DCA672100DC
:10356000BC310D602100C03108602100C4310B6006
:1035700021000635CC310D602100083DC8310D60B9
:103580002100D0310A602200D43210602200D832EB
:10359000136022000227E032210017604222DC3152
:1035A0000A6021001B3DE4310D602100E831086014
:1035B0002100EC310B6023000521F4331960230056
:1035C000F0331A602300183290331A6023009433CA
:1035D000186023001E3A98331A60AF23DB00236083
:1035E000644BFA262363644B644DE360644BF03113
:1035F000A3642300FF31FC33B600A16021611E608B
:10360000A5627325E5656D3D6565A56596255D4AF1
:10361000AD00E264666258606766A566002709250A
:10362000A767E566584F594D606720002567E26738
:103630003A6015279C30676007001A203860200028
:10364000A0300700212038602000A83007004C4837
:1036500038602000F830066026006427A436376002
:1036600026005F3FAC3637602600033FB036376038
:103670002600C637B436376026000027B8363760D4
:1036800038269E60424E96205E64424E5A66DE6147
:10369000414E9A645E62F53EFF3E9E621E269A6728
:1036A000354A8000DE661F675F67DD651D6618624C
:1036B000DA67BE23394A5B00E250394BD8382350D1
:1036C00004302250C4225200A350C623E4205B00E1
:1036D000E1500433334AE1503349344BD16034492B
:1036E000800019503349E938FF3819503249043005
:1036F000195032493248D16132491163324951631C
:103700001900F4310860CE20304940001160304982
:10371000195019002F48F83108602F49D1658221CE
:103720002E4A89005A501A002D490832D1671A00D2
:103730002C49B432116088212B4A89005A501A0052
:103740002A49883211602A4ADA6408F00DF801200B
:1037500008F092F9F8BDC0460004FF1F1C65FF1F6A
:103760000070FF1FE844FF1F4A0AFF1F3A070000CE
:1037700080C3C9019A020000DC0500006A1800003D
:1037800050C3000088130000F009FF1F204E000006
:103790006509FF1F68100000C409000040420F00C7
:1037A00010270000FC00FF1F791CFF1F0000FF1FF7
:1037B000CD2CFF1F5D30FF1FF52EFF1F3920FF1F8F
:1037C0002927FF1F5520FF1F0122FF1FC51FFF1FB5
:1037D0004D29FF1F352AFF1F9119FF1F5928FF1F71
:1037E0007D25FF1F8925FF1FC51EFF1F7D1FFF1F92
:1037F0003D1EFF1F0223F0B501245F4D5F4E2B706D
:103800005F4B91B01C705F4F039333680021200021
:10381000FB7006F0E5FD200006F0DCFC002398427A
:1038200005D0FA78552A02D0332A00D097E03360C9
:10383000042006F03DFF07F0C7FFFFF75DFE08F02C
:1038400023F91F22012400214F4B10AE1A704F4B59
:103850001C704F4B19704F4B19689143163A0A432D
:103860001A60602219689143403A0A431A6008F0CE
:103870006BF908F0C9F9C120FF21474B80001A58A5
:103880008A431A50C522920098588843BF39014391
:1038900099509858414908408021C901014380202E
:1038A00099509958C0050902090A0143995080218D
:1038B0003B48490107F038FF0323220039490194AE
:1038C0000093394807F0A8FE2C22384905A808F0D3
:1038D000CBF805AC61782078023406F09BFCA64258
:1038E000F8D1334C334B226803201A40A023DB026B
:1038F00013432360802322689B04134323602268C0
:103900002D4B1A4080239B03134323602B4A2C4BDF
:10391000934200D8012008F05FF908F0DDF8802319
:103920002268DB0413432360287807F0F5FF039B2C
:103930001878C0B208F018F808F0B6F82149042049
:1039400008F00AF806F080FE00F03EF800F0E6FD10
:1039500000F08EFE00F008FA002011B0F0BD0093D8
:103960002100184A042007F087FF8023DB059C62B2
:10397000FFF76CFD5CE7C0464A0AFF1F34F00040C9
:10398000E844FF1FA862FF1F480AFF1F490AFF1FE4
:10399000680AFF1FBCF0004000E100E0FF00FFFFED
:1039A000EC44FF1F7057FF1FEC54FF1F18BC0011A1
:1039B00014F00040FF7FF8FFFFFF9FFF0080FF1F14
:1039C0000070FF1F3B000108002210B511001120FC
:1039D00007F032FF10BD0000F8B500230926364F6E
:1039E000364C3B62E3681120B343E36008F064F8AF
:1039F000112007F071FE112007F0CEFF402322684E
:103A000010251343236080236268DB021343636045
:103A10008023A26802211343A360A368284A0820D8
:103A20001340A3608023A2689B0113430122A3607B
:103A3000236CAB432364236C1343236480231B0157
:103A40003B62226B1F4B1A402263626B1A40626317
:103A5000A26B1A40A263E26B1340E363E3681A4A65
:103A60001340E36006F0D6FB0121082006F0E6FCD7
:103A70008023164A5B00516C11200B43536407F0FE
:103A8000CBFEFD21C720124B124A89005A50A36B6E
:103A900080002B43A363E3680F4A3343E3600F4B7B
:103AA00019581140802212020A431A5080229205AE
:103AB0001A600B4B5D63F8BD00F000403CF0004025
:103AC000FFFFDFFFEFFFEFFFFFFF7FFF003800404A
:103AD0000000FF1F5118FF1FFF00FFFF00E100E083
:103AE0000000054070B5284C238C002B23D0228A7F
:103AF000002A21D1DA0023826382A382E382238316
:103B00006383A383E38322606260A260E2601F4D4F
:103B10001F4A6420EB8093420AD8FA220020D20088
:103B2000934205D91B4A0A21981807F045FDC0B2F7
:103B300000232872238470BD0720E11CCA7F013254
:103B40000240CA7705D10325201DC17F01312940DC
:103B5000C17708325200A352002321001A00088ABC
:103B600001321B180231082AF9D1221DD27F92009E
:103B7000A350626823689B18A2689B18E2689B1890
:103B80005B099BB2C3E7C046E861FF1F9062FF1F5D
:103B9000B70B000030F8FFFF30B503A804880B20F6
:103BA000002C0ED14968074D087849780902014375
:103BB0000A20A94205D1012120001980024B1B7A5D
:103BC000137030BD192A00009062FF1FF7B5150071
:103BD00008AA16884A680F4F1478527812022243B6
:103BE0000A24BA4214D10122DBB2019200962A00C3
:103BF00007F07AFC041E0BD1074B1B68002B07D083
:103C000068782A78000210434242504101309847B8
:103C10002000FEBD022900001462FF1F30B50125FF
:103C200003790400BFB02B4211D00A49408806F046
:103C3000C7FF28420BD0084B01A95B8D4D800B803C
:103C4000064B00221B7A60880B7104F0ABF83FB082
:103C500030BDC0460C62FF1F2041FF1F9062FF1F56
:103C600010B50549054806F061FF0421044A0548DE
:103C700006F01EFF10BDC0460C62FF1FFFFF0000D4
:103C800044BC00112041FF1F10B5024804F00CFF96
:103C900010BDC0461D3C0011012303700B4B1A7A66
:103CA0004270022282709A78C270DA78027103221E
:103CB00042711A7982715A79C2710C2202729A7910
:103CC0004272DB7983720B207047C0469062FF1FFF
:103CD000022310B50370013B43700533837010332A
:103CE0000371443B43712A3383714433C37100230E
:103CF0000372064B04001B8843720A30FFF7CCFFA7
:103D0000831D0A30C0B2E37010BDC0469062FF1F31
:103D100010B5142007F0C0FC124B142200211860CB
:103D200007F0FAFE002007F0BFFC012007F03CFE80
:103D3000022007F079FD032004F05AF9042006F070
:103D40006FF9052003F098FB062004F065F80720C2
:103D500001F062FA082006F08BFE092001F03CF821
:103D600010BDC0461862FF1F07F036FE012007F0A5
:103D70005BFE07F051FE0000094B10B504009842AD
:103D800005D0012904D12000064906F0CFFE10BD60
:103D90000229FCD1013904F045FE0028F3D0F6E7F2
:103DA000FEFF00003E62FF1F70B50D7A100004AAEE
:103DB0002C00168810221440154220D1002E20D14C
:103DC0000A78022A18D14A68517815780E4A0902F1
:103DD0002943914205D00D4A914209D01C800A2402
:103DE00004E014220A491A8007F03EFE200070BD4C
:103DF0000C2208491A80F7E71C800124F6E7082402
:103E0000F4E70B24F2E7C046F3FF0000F4FF0000E4
:103E10007443FF1F20BD001110B504000749084876
:103E200006F084FE074804F07FFD0020E40704D577
:103E30000721054A054806F03BFE10BD3E62FF1F04
:103E4000FFFF0000793D001188BC00116441FF1F95
:103E500000B50C4BBFB01A780B4902A800F0C2FCA9
:103E60006B4680B2D880002809D06A46074B01A96A
:103E70001B889380064B0022188803F093FF3FB005
:103E800000BDC0461C62FF1F1D62FF1FBE41FF1F19
:103E9000C842FF1F00B50C4BBFB01A780B4902A8EF
:103EA00001F0C6FE6B4680B2D880002809D06A4671
:103EB000074B01A95B8D9380064B0022188803F005
:103EC00071FF3FB000BDC0464662FF1F4762FF1F43
:103ED0006441FF1FC842FF1FF7B50E00377A1C0070
:103EE00008AB11003D001A8820231D401F423CD121
:103EF0003378022B3BD173681F785B781B023B43FE
:103F00001E4FBB4208D01E4FBB4214D01D4DAB42CA
:103F100021D00A252800FEBD002A2AD1142C2AD837
:103F20002200F06807F0A0FD174B1C70012CF1D99E
:103F3000FFF7B0FFEEE7002A1BD1202C1BD8220090
:103F4000F06807F091FD114B04211C70104B18789C
:103F500007F042FCDEE7E3B20124009201940A007C
:103F6000310007F0C1FA0500D4E70825D2E70125A2
:103F7000D0E70B25CEE70D25CCE7C046F3FF0000C8
:103F8000F4FF0000022900004662FF1F1C62FF1FB1
:103F9000C862FF1F332310B5040003700A220749CB
:103FA000013007F061FD064B0F201B681A0AE3720F
:103FB00022731A0C1B0E6273A37310BD9062FF1F55
:103FC000B862FF1F30B5012503790400BFB02B4252
:103FD00013D00B49408806F0F3FD28420DD06A4605
:103FE000084B02A81B889380FFF7D4FF6B46D8804C
:103FF0000022608801A903F0D5FE3FB030BDC04665
:104000003E62FF1FBE41FF1F10B5024804F04CFD89
:1040100010BDC046C53F001170B5160004AA148833
:1040200005AA15784A685078117800022A4A084390
:10403000801805284BD807F097FD03131E29343F3D
:104040000720032C0BD80422121BAA4200D92A00F5
:1040500022491A803000091907F006FD002070BDC2
:104060000720112CFBD81222121BAA4200D92A00C9
:104070001B491A80EEE707200E2CF0D80F22121BE6
:10408000AA4200D92A0017491A80E3E70720032C27
:10409000E5D80422121BAA4200D92A0012491A802C
:1040A000D8E70720032CDAD80422121BAA4200D931
:1040B0002A000E491A80CDE70720032CCFD804220E
:1040C000121BAA4200D92A0009491A80C2E700221D
:1040D0000A201A80C3E7C046DCD5FFFFD3BC00111D
:1040E0006462FF1FC3BC0011BEBC0011B9BC00114B
:1040F000B4BC001110B50D21024A034806F0D8FCEB
:1041000010BDC046A8BC0011D441FF1FF0B500246B
:10411000274E85B03000B47100F0E2F8254D264BF3
:10412000EA89297C9A422FD10423300003AA00F0A7
:1041300057F90400300000F011F90123B371002C8D
:1041400034D16B4699892B68C9BA4B4329891B4ADC
:104150001B145B1853806B46D9896B6849BA89B2C6
:104160004B4369891B0C5B181548191C1BB2834211
:1041700000DD011C0B0400D5002113889180013360
:104180001380200005B0F0BD0227220003AB3000F1
:10419000009700F0F7F80E230400297C012230007C
:1041A00000976B4400F0EEF80443C3E71C00E8E717
:1041B000AC42FF1F7862FF1F830500009062FF1F63
:1041C0000F27000073B5234E300000F089F8224D10
:1041D00007236A463000297C00F002F90400300011
:1041E000002C33D16B461B787F2B2FD800F0B6F80C
:1041F0006B46D878F02302041B031A406B469B8859
:1042000016495BBA9BB21A432B68000953432A89AB
:104210001B0C9B184B806B465A789B7812031B0132
:104220001A436B68024353436A891B0C9B180C4862
:104230001A1C1BB2834200DD021C130400D50022AD
:104240000B888A8001330B80200076BD00F086F851
:104250000124F9E7AC42FF1F7862FF1F9062FF1F45
:104260000F27000070B5114C237C002B0FD0382B8A
:104270000ED10F4D280000F033F8CC23AC222800DB
:10428000217C9B0100F0F4F8280000F067F870BD75
:10429000084BE2899A42FAD1054D280000F020F837
:1042A00000222800217C00F0C5F8EDE77862FF1FAE
:1042B000AC42FF1F8305000010B5084B1A7C002A92
:1042C00009D05B69002B06D09847041E01D0FEF789
:1042D00097FE200010BD0124F9E7C0467862FF1F59
:1042E00070B5C17905000C00631E9C411A4BE402B5
:1042F000E41849000460C9B2007906F0D5F8E979FC
:10430000687949000131C9B206F0CEF8E879093080
:10431000C0B207F041FB0023E36661332360AA7952
:104320005B3B002A0ED022689A43023B1343236072
:104330000A23E3610733236200232363A36301336A
:10434000E36370BD22689A4302231343236046232C
:1043500063610633A361EFE70050004070B50025AC
:1043600004000368DD66C0790930C0B207F0A4FB21
:104370002900207906F034F82900607906F030F839
:1043800070BD0000F8B51E0006AB1D780023046860
:104390001700E366616007F0A7FA01238022E36655
:1043A0002B0027615200013B08D207F055FB082083
:1043B0000A4A1168002D03D12800F8BD2261F2E7F6
:1043C000236F034203D02369013D33700136136824
:1043D0005B1A032BEED90125EEE7C0466008FF1FEC
:1043E00070B51C00002305681600EB66696007F0D5
:1043F0007BFA01238022EB6623005200013B08D2A6
:1044000007F02AFB08200A4A1168002C03D120007B
:1044100070BD2A61F2E72B6F034203D02B69013C88
:104420003370013613685B1A032BEED90124EEE7D3
:104430006008FF1F002370B504681500E366616023
:1044400007F052FA0123E366256107F005FB80209F
:10445000064A80001168636B034205D113685B1A3A
:10446000032BF8D9012070BD0020FCE76008FF1F76
:1044700070B51D00002304681600E366616007F054
:1044800033FA0123E36626610F33626B1A42FCD0D4
:104490002B0A23611023626B1A42FCD0EDB2256116
:1044A00007F0DAFA8020074A80001168636B034244
:1044B00005D113685B1A032BF8D9012070BD0020C9
:1044C000FCE7C0466008FF1F70B51E0000230568AA
:1044D0001400EB66696007F007FA0123A619EB6682
:1044E0000F33B4420ED107F0B7FA80200A4A800099
:1044F00011686B6B03420CD113685B1A032BF8D95C
:10450000012070BD21782961696B1942FCD001340A
:10451000E7E70020F5E7C0466008FF1F10B5084C2C
:10452000E368002B08D18022064B52021B689B18BF
:104530006360054B1B68236007F0E6F8A06010BDC0
:10454000B862FF1FC8F00040CCF0004070B5184AB8
:10455000936A916A9942FBD116498A689A421FD39D
:104560009A1A8B60144B0126186893B2D202D20EAD
:104570004343424300204C681B0A1B1912029B183C
:104580000E4C0A684B60551CA3420CD8002801D081
:104590004B600A600A4A136008680A4B186070BDD5
:1045A000581E821ADDE7084A30009B182A00EAE705
:1045B00000F00040B862FF1F140AFF1F40420F00C6
:1045C000C8F00040CCF00040C0BDF0FF70B51F4CFB
:1045D00023793F2B01D93F2323711D4B22791A7078
:1045E0001878C0B206F0F0FF18231A491A4A0B8057
:1045F0001A4913800B805380A379194980200B80BE
:104600000C21938001334B43164D191C000183424A
:1046100000D9011C2980D1806379002B11D101338D
:104620006371237A012B01D8022323726279237AE2
:104630000D4853430A21584306F0BEFF0B4D286036
:1046400070BDA02BEDD9A023EAE7C046AC62FF1FE6
:10465000480AFF1FC642FF1F9444FF1FC442FF1FAA
:10466000C242FF1FC042FF1F710200009C62FF1F79
:10467000F8B514210020FEF7B1FE114C011E114DBA
:1046800009D10C22104BC1CBC1C4280007F044FA59
:10469000FFF79CFFF8BD0C2220000C49FEF772FECC
:1046A0000C2802D0084B43CB43C40C2228000849F5
:1046B000FEF768FE0C28EBD00C220021E5E7C0468F
:1046C000AC62FF1F7862FF1F14BD0011FC0C0000DC
:1046D000F50C0000F0B51D4C8022A5440400882094
:1046E00069465201400506F0FFFF902212016A441C
:1046F0001300200032C832C316C816C38023144CDE
:10470000144FA6689B033343A3603B6007F07CF91A
:104710008823A0685B05C01807F0C6F80025882329
:1047200029008022A0685B05C01840196944520026
:1047300007F0B2F980230135FF355B019D42EED1D0
:10474000A6603E60044B9D44F0BDC046FCEFFFFFF9
:104750000444FF1F9808FF1F04100000F0B5040078
:1047600087B0002825D0684607F0AEF81B4C022819
:1047700006D106226946200007F01EFA002816D04E
:104780006946002301250F262F00E25C0133100942
:104790001030874038002F00324097403A000243E3
:1047A0004A610439062BEFD16846FFF793FF07B043
:1047B000F0BD182269460A4806F096FF6A46A30033
:1047C000D358013305D01822FF21684607F0A4F919
:1047D000EAE70134062CF1D1E9E7C0466509FF1F7D
:1047E00000090011F0B5002504000E0085B0AA42B2
:1047F00000D186E04B1C087801934B788978377993
:1048000009021943F3783F061B040B431F43039728
:1048100020706570252800D196E033D8112813D870
:1048200007F05AF869002B012B012B012B01AA007C
:10483000B800B1002B012B012B012B012B012B0107
:104840002B012B0105012501232800D1DEE0DB2807
:1048500000D034E1042A00D8ACE01025052A05D0A8
:10486000551F2A003800711D07F0FEF8052231009F
:10487000200007F0F9F82A003900601D07F0F4F86D
:1048800005353EE0562859D010D8332800D19DE098
:10489000552839D02628DAD19F4B29001322180039
:1048A0001D0007F039F9FEF7ABFB5CE0712800D181
:1048B00077E0722800D180E0602800D18BE0DC280E
:1048C000C5D1022A00D875E07378BFB26370B3789F
:1048D000A370032A05D0033A390092B2F01CFEF708
:1048E0008BFC10223900E01CFEF74CFDC51C002893
:1048F00007DA60705CE00C222000884907F0B4F809
:104900000C25280005B0F0BD013A854D0C2A13D8BE
:10491000002A0AD02800019907F0A6F8FFF756FEF2
:104920000C2228007F49FEF767FC29000C22601C3E
:1049300007F09AF80D25E4E70C22EBE7784D7A4B67
:104940002A0043CB43C2E9E7013A734D0C2A11D840
:10495000002A08D00199280007F086F80C222800C8
:104960007249FEF749FC29001322601C07F07CF80D
:104970001425C6E70C22EDE705226D49601C07F0FF
:1049800073F80625BDE712226A49601C07F06CF82F
:104990001325B6E708226849601C07F065F8092569
:1049A000AFE77178F02905D8644B188801F09CFDB9
:1049B0000225A6E7FF236370FAE7614B012A03D0C3
:1049C00072789A706270F3E79B78F4E72000FFF743
:1049D000E1FA050095E7013A594B5A4D072A10D8DC
:1049E000002A10D0012128005970019907F03CF8E5
:1049F00001F058F829000722601C07F035F8082557
:104A00007FE70722EEE700225A70F3E7042A04D971
:104A10004D4D2F6006F078FEA860FFF797FD042249
:104A2000039003A9601C07F01FF8052569E7474DAF
:104A3000062A15D906222800019907F0BDF800289A
:104A40000ED006220199280007F00EF806224049F0
:104A50002800FEF7D1FB0123394A91780B4393706C
:104A600029000622601C06F0FFFF072549E7012AFE
:104A7000A0D07078FFF772FE9AE7012800D0E6E632
:104A8000931E344F132B04D87378002B09D100F0F8
:104A900015F9314B39001D78601C6A1E06F0E4FFE1
:104AA0002FE7551E2A000199380006F0DDFF2B493B
:104AB000AAB23800FEF7A0FB00F038F9E9E7DA28DF
:104AC0001DD1042A00D875E7082A15D9B37972795F
:104AD0001B021343F27912041A43337A1B06134361
:104AE0003B603B68052231002000039306F0BCFFC9
:104AF0000422601D03A950E7FE236370F1E7DE285E
:104B000000D057E7511E012A01D10025F9E601988E
:104B100000F0AEFFF9E7C0467862FF1F20BD00112C
:104B2000AC62FF1FFC0C000014BD0011F50C00006E
:104B30008462FF1F6462FF1F0844FF1FC842FF1FFB
:104B4000A862FF1F6543FF1FB862FF1F6509FF1FB3
:104B5000ADAC0000A964FF1FA764FF1FAEDE00001C
:104B600070477047020010B5094B0A32094C92B2E7
:104B7000DA815A8298811882207802F01BFB042285
:104B8000054B012120781A7006F026FE10BDC046A4
:104B90009243FF1FF264FF1FF164FF1F013870B5DD
:104BA000042809D806F0E0FF030928081200234B67
:104BB0000221187806F010FE70BD204B08211878ED
:104BC00006F0F2FF00221E4B1A72F5E78022002445
:104BD0001B4B1A4D52001A8108211A682878DC7282
:104BE00006F012FE2100287806F0A6FF012000F052
:104BF0005FFE00F057FFDFE7104B0821187806F042
:104C0000D3FF1048FFF764F80F4B104A9B79002040
:104C100093800F4A13808022094B5200D8721A8168
:104C200000F046FE00F03EFF0A4B9B78002BC3D0FD
:104C3000094A136006F068FFBEE7C046C862FF1F5E
:104C40009C62FF1FD142FF1FAC62FF1F9444FF1FF5
:104C5000C242FF1FA862FF1F34F0004010B50129B7
:104C60000BD1012809D1054B1B78002B05D026223A
:104C7000034B04485A72FFF775FF10BDCA64FF1F4B
:104C80009C62FF1FC40900000300F0B50A4D8E1896
:104C9000B14202D152008018F0BD0C782F6824096F
:104CA0003C5D0F271C700C7801313C402F683C5D47
:104CB0005C700233ECE7C046BC42FF1F0D22124B72
:104CC00010B51A700C23114C11492370093A033B9B
:104CD0001048637006F0C8FE2D2301220E490F48CC
:104CE000A371FFF7D1FF01220D49FFF7CDFF01228C
:104CF0000C49FFF7C9FF030000200B4902001870A0
:104D0000FEF77AFA10BDC046C664FF1FA764FF1FF6
:104D1000D3BC0011A964FF1F6709FF1FAE64FF1F0A
:104D20006609FF1F6509FF1FAEDE000070B5124C5B
:104D3000142220001149FEF725FB431E104D132BB2
:104D400017D8AB78002B14D0431C2B7009236B7041
:104D5000002300190370287829000130C0B206F042
:104D60002BFD297822000139C9B2002005F0BEFDD3
:104D700070BDFFF7A3FFEEE7A964FF1FAEDE0000E2
:104D8000A764FF1F10B5114B1A781870002A0ED0B7
:104D900000280BD10E4B1A78062A07D85423D3408B
:104DA000DB0703D50B4B187802F004FA10BD00287E
:104DB000FCD0074B1B78012B02D0033B022BF5D80C
:104DC000044B0121187806F007FDEFE7CA64FF1FC6
:104DD000F164FF1FF264FF1F70B54A4E4A4A4B4907
:104DE0003070012005F00EFC00F0C0FEFEF708F95F
:104DF00006F032FD032246494648FFF745FF2D24C1
:104E0000030004221C7044490130FFF73DFF3023AA
:104E10000470424D424C437083702E3B06222000AA
:104E20004049EB87FEF7AEFA062813D0200006F0C3
:104E30004BFD022809D00321200006F0A5FD8D239B
:104E4000E3706E3B237119336371062220003549EC
:104E5000FEF7D2F9344B1B68FC335C64FFF766FF46
:104E60000020FFF78FFF314C314A0121314B12787E
:104E7000207802F061F9304A304B12780021207816
:104E800002F05AF901222E4B1A702E4BDB78552B6B
:104E900031D12D4B3B325A722C4B2D4AAB81EA81DA
:104EA0002B826A822021307806F026FE01204042C3
:104EB00005F068FD0120404205F004FEFFF71AF9F5
:104EC000FEF7CEFE00F0B2FC01204042FEF7A4FF48
:104ED000012006F029FEF02001F0EAFA01213078E5
:104EE00006F07AFC307802F0C1FA1A4806F064FD48
:104EF000FEF772FD70BD6422174B5B7953431A00B5
:104F00000A32CBE7C862FF1F614B00115D4C0011F4
:104F10000844FF1F6462FF1F8462FF1F9243FF1F4C
:104F20006509FF1FADAC00001C65FF1FF264FF1F89
:104F3000F042FF1FD142FF1FC664FF1FA764FF1F7F
:104F40009864FF1FA862FF1F9C62FF1FC409000036
:104F5000CE090000CA62FF1FAC62FF1FF8B50A004D
:104F600020230D001A40194263D05E4B1B78002BA2
:104F70005CD0FFF7EBFA5C4B5C4C5D4E9968626865
:104F8000737A8A1ADB039A4202D36160FEF724FD2A
:104F9000327A217A531EDBB2994205D1FFF762F9CA
:104FA000002000F0B5FD15E09142F9D300272772EB
:104FB000FFF782F9A37ABB4202D0A772FEF792FDF7
:104FC000012000F0A5FD4B4F3800FEF781FE3900AF
:104FD00006F072FC637A002B25D0013BDBB26372D2
:104FE000002B20D1444BDB78552B01D106F08CFDF2
:104FF000E37A002B12D00023A27AE3729A4202D005
:10500000A372FEF76FFD3D4A3A4F13883800013313
:105010001380FEF75DFE390006F04EFC64237079C4
:105020005843FFF79FFD237A013323722020684005
:10503000F8BD0BB2002B0ADA314B187806F0DCFC15
:10504000002801D006F0F8FA80200002EFE70224E1
:10505000214206D0254B01201A72FFF793FE200053
:10506000E5E70B071ED5FFF771FA1F4B1F49204CD0
:1050700098684A68637A821ADB039A4202D34860CE
:10508000FEF7AAFCFFF718F9FFF7ECF8012000F093
:105090003FFD00F0E5FB2368DB0701D5FEF7B4FF19
:1050A0000820C4E7CB0609D5FEF71CFD0D4B1B7885
:1050B000002B01D1FEF7E8FD1020B8E701242142C2
:1050C00007D0104800F06CF806F02EFC00F006FD4A
:1050D000C5E70424080020402142A9D0FEF7B8FE0D
:1050E000BDE7C046CA64FF1FB862FF1F9C62FF1F76
:1050F000AC62FF1FD142FF1FA862FF1F9062FF1F1B
:10510000C862FF1FB442FF1FF0B51B4B1B4F1B882B
:105110003A8804001A4E1B4D85B09A420DD8328849
:105120009A420AD3184B1A882B889A4205D1174AFB
:10513000174B12881B889A421BD0052001F00EFAEB
:105140003B8802AA13803388019053802B88114D2D
:1051500093800F4B02A91B88D3800F4B2A781888A5
:1051600002F02AFF0D4B08212878019A1C7006F0E6
:10517000A3FA05B0F0BDC0469664FF1FC642FF1FEC
:10518000C442FF1FC242FF1F9464FF1F9264FF1FAF
:10519000C042FF1FF264FF1FC842FF1F9064FF1F41
:1051A00013B50C4B1C78002C11D1002801D00A4BF0
:1051B00018600A4A0A4B11780A4A10780A4A019282
:1051C0000A4A0092002205F089FA200016BD112437
:1051D000FBE7C046F164FF1F8C64FF1FF064FF1FF4
:1051E000E064FF1FF264FF1FCC64FF1FD064FF1F49
:1051F00010B5064B12201B78052B06D1044B132249
:105200001988044B187801F085FB10BDF164FF1F6D
:10521000C842FF1FF264FF1F10B500240122114B8A
:1052200052421870104B1C70104B1A8002F01EF97D
:1052300004220F4B21001A700E480C3206F00CFAB3
:10524000102221000C4806F007FA07220B4B1C60C5
:105250000B4B1C700B4B1C700B4B1A700B4B1C70C8
:1052600010BDC046F264FF1FF164FF1FC842FF1F5C
:10527000F064FF1FE064FF1FD064FF1FCC64FF1FBA
:10528000A664FF1FA564FF1FCA42FF1FA464FF1F7F
:10529000F8B5174C0600257806A814240078052DCB
:1052A00023D1B41F134FA5B21824BD421DD88D1FA2
:1052B000ADB2BD4219D8FA256D00AA4215D21D0023
:1052C0000D4F0A3DADB2BD420FD80C4C26800C4CA0
:1052D00021800C4900240A800B4A1380FFF714FF39
:1052E0000A4B0421187806F05FFC2000F8BDC04688
:1052F000F164FF1F790C0000750C0000C642FF1F0F
:10530000C442FF1FC242FF1FC042FF1FF264FF1FC3
:10531000F0B50BB20D0089B0002B00DB70E1A44E9C
:10532000307806F069FB041E50D00378A22B00D120
:1053300022E1D02B1AD0912B45D143780E2B42D1AC
:105340009C4B82889A423ED19B4A83681278052AF8
:1053500039D1032018567F2835D0984B1B68002B75
:1053600031D05B68002B2ED098472CE0807807283E
:1053700029D806F0F9FB0428183F3F74A8D86378B1
:10538000002B0CD101218C4B19708D4B1A78002AFF
:105390005BD08C4B307801F0CFFE002855D007222F
:1053A000854B1A7051E061780029F8D1E378002B21
:1053B00011D0854A854B1278307801F0BDFE6070BF
:1053C0006378002BEBD1200006F036F98020000234
:1053D000684009B0F0BD784B1B78022BF3D0012157
:1053E000307806F001FB0028EAD10121307806F080
:1053F000F3F9E5E76378002BD1D16F4F032807D18C
:105400003B78052B02D101333B701EE00223FBE702
:105410006F4B1A886F4B0293002A0BD01B78002B1E
:1054200003D00121307806F047F93B78062B04D1F0
:10543000013BE9E7029B1A70F7E7042B41D10121F8
:10544000029B3078197006F0C7F95C4B1B68002B83
:10545000B9D01B68002BB6D0574A107884E7637820
:10546000554F002B27D10622211D5B4806F0FCFA80
:1054700062895A4B5A491A80A2895A4B1A80E38989
:105480000B800521397058490A80584A1380228AB6
:10549000574B1A80574B1B78012B09D11F2001F065
:1054A0005DF8FA22920042430421307806F004F9B4
:1054B0000022484B75E7312B00D070E70022454BA6
:1054C0001A700323A0E706220021434806F0C4F81F
:1054D0000023454A04211380444A30781380444A0B
:1054E000138006F061FB0821307806F05DFBA3799C
:1054F000083B5A425341304A03331370304B1B78F8
:10550000002B06D0334B30781A78002A06D001F0F1
:1055100051FE0122314B52421A8096E70121197047
:1055200006F05AF9F5E70821307806F03DFB63787C
:10553000002B00D047E72C4B2D4F0293E388029AB3
:1055400004211380294B307803932389039A138015
:1055500063893B8006F048FA002800D033E7264BE9
:105560001B68002B00D12EE7039902983A8809881E
:1055700000881B68984726E74379132B00D022E761
:105580000389012B0AD11D4B1B78022B06D1082160
:10559000307806F009FBFFF72BFE14E7052000F03A
:1055A000DDFF08210200307806F086F80BE7C046E0
:1055B000F264FF1F05140000F164FF1F8C64FF1FDD
:1055C000F042FF1FD142FF1FC664FF1FA764FF1FE9
:1055D000C864FF1FCA64FF1F9964FF1FC842FF1FF2
:1055E000A064FF1FA264FF1F9664FF1F9464FF1F47
:1055F0009264FF1F9864FF1F8864FF1F9064FF1F61
:105600008020C001014200D0E2E6CB0731D5324B09
:105610001B78002B1DD0314E05AC3378052B1AD1E9
:10562000023B23702E4B21001B7823722D4B1B78DD
:1056300063722D4B187801F023FD002809D0072054
:105640002A4B30701B68002B03D01B68002B00D046
:1056500098470120BCE60E20254B06221B782549E1
:105660002370254B1B78637002ABC01806F0FCF961
:10567000D8E7022308001840194209D0174B1B78BD
:10568000052B03D11D4B188806F046F802209FE633
:105690000424214203D0FFF737FD200098E60823B9
:1056A00008001840194200D193E6154B1C78012CD4
:1056B00003D0022C0DD008208AE6124B124A13495F
:1056C00013481B881288098800880094FFF7E0FDC2
:1056D000F1E7FFF78DFDEEE7CA64FF1FF164FF1FDE
:1056E000CA42FF1FA464FF1FF264FF1F8C64FF1FE8
:1056F000A664FF1FCB42FF1FA564FF1FC842FF1F08
:105700009064FF1FC042FF1FC242FF1FC442FF1F21
:10571000C642FF1F10B502A804880B20002C10D130
:10572000496808784978090201430C48814209D147
:10573000022119800A4B59881170DB7800205BB276
:10574000537010BD074C0A20A142FAD102211980E2
:10575000034B998811705B79F0E7C0466E2A000010
:105760009062FF1F6F2A0000F7B5150008AA16887F
:105770004A680F4F14785278120222430A24BA4220
:1057800014D10122DBB2019200962A0005F0ACFE92
:10579000041E0BD1074B1B68002B07D068782A78B2
:1057A0000002104342425041013098472000FEBDA4
:1057B000022900000465FF1F30B5012503790400AC
:1057C000BFB02B4225D01449408805F0F9F9284292
:1057D0000CD0124B01A95B8D00220B8002234B8061
:1057E0000F4B5B888B80608802F0DCFA0D49608883
:1057F00005F0E6F9C0070CD50B4B01A91B88002268
:105800000B8002234B80064B9B888B80608802F0C4
:10581000C9FA3FB030BDC046FC64FF1FF442FF1F11
:105820009062FF1FF464FF1F4E43FF1F10B5074C2B
:105830000749200005F07AF92000064905F076F9BD
:105840000721054A054805F033F910BDFFFF0000A8
:10585000FC64FF1FF464FF1F40BD0011F442FF1FF2
:1058600010B5024803F020F910BDC046B957001129
:105870000221430888400B400A31084003430E20B0
:10588000024AD17881430B43D37070476543FF1FB1
:10589000064A1379410705D580210B438001137116
:1058A000907170477F210B40F8E7C0466543FF1FAA
:1058B000054A5378002803D080210B43537070476A
:1058C0007F210B40FAE7C0466543FF1F0F21114BB4
:1058D000DA780A40DA70502810D901310A43DA70B8
:1058E0002022D9780A43DA704022D9780A43DA7044
:1058F0008022D97852420A43DA7005E03C28EFD87A
:105900002828F1D81428F3D80122D9780A43DA706C
:105910007047C0466543FF1FF8B57F23324D040032
:105920006E789E43314B984205DD76232B70363BD3
:1059300033436B70F8BD2E4B984203DA58232B701B
:105940001433F5E783B21A0000215F32294892B27E
:10595000294F297082422DD9A9708C4203DA5B420B
:105960001CB220232B70053420B20A2105F024FE3E
:1059700004B2FA239B009C4233DB80232A785B42EB
:1059800013432B706421200005F016FE0A2100B29B
:1059900006F09AF809B22A787B5C13432B700A212F
:1059A000200005F009FE0A2100B206F08DF809B2C8
:1059B0007B5C0AE08022AA70002CDADA5B421CB21F
:1059C00020232B705F23092CE9DC1E430A212000D1
:1059D0006E7006F079F809B2AA787B5C1343AB705D
:1059E000A8E7632CCEDCEDE76543FF1F1B4E0000EC
:1059F0001DFCFFFF2A0800006ABD00117F23F7B5D8
:105A0000194FCD013E7904009E433E71EDB26328EB
:105A100006DD093B33433B7140231D437D71F7BDD8
:105A20000300093304DA582333433B716C23F4E752
:105A30000E4B019300280BDA0423444224B23B713D
:105A40000A21200006F040F8019B09B25B5CE4E704
:105A50000928F5DD0A2105F0AFFD019B00B21B5CB2
:105A60001E433E71ECE7C0466543FF1F6ABD00114F
:105A7000F8B50A4F05003B780E00002B0CD0084CFF
:105A80002000FEF72DFC33002A0020003978FEF7B5
:105A90001BFD2000FEF762FCF8BDC0461065FF1F2D
:105AA0006C43FF1F70B50A4E0A4D072231002800D3
:105AB00006F082F8002809D0074C310007222800A0
:105AC00005F0D2FF08212000FFF7D2FF70BDC046CD
:105AD0006543FF1F0965FF1F0865FF1F7F2210B583
:105AE0000A4B59789143033A1A70103A0A435A7094
:105AF00078220E219A70DA788A43DA7006221A71B7
:105B000030325A71FFF7CEFF10BDC0466543FF1F0C
:105B100010B5002824D0134C0A210223E05E05F0C2
:105B20004BFD00B2FFF7F8FE0423E05E642105F0B0
:105B300043FD012100B2FFF761FF207AFFF7C6FEA7
:105B40000320FFF795FE0020FFF7A2FE064B187812
:105B5000053843425841C0B2FFF7AAFEFFF7A2FF43
:105B600010BDC0469062FF1FF164FF1F70B5002496
:105B7000094D2800AC71FEF7B3FB10233E2128002D
:105B8000064AFEF7A1FCA04200D13E34044B280097
:105B90001C70FEF7E3FB70BD6C43FF1F5ABD001184
:105BA0001065FF1F0200F0B501270A480A4E511880
:105BB0008B1A002B00DCF0BD0824157843086840E0
:105BC00038404000805B013C58406D08002CF5D106
:105BD0000132EDE7FFFF00007ABD0011F0B50025AE
:105BE0000F269D4200DBF0BD4C5D07094440344068
:105BF000A400A05801357840F3E70000F0B589B063
:105C00006A460D000B000F27110010351C78013378
:105C1000260024093E40167054700232AB42F5D182
:105C20002023024AFFF7DAFF09B0F0BD80BD001162
:105C3000F0B54E780B7889B036020C001700019051
:105C40001E43012A61D9954B9E4200D877E001336B
:105C50009E421CD1062A17D1CA788B7812021A43A9
:105C60000B791B0413434A7912061A438C4B5A6171
:105C700000221A705A808B4A5A608B4A9A608B4A6B
:105C8000DA60002009B0F0BD88225205EEE7884BAB
:105C90009E423CD182498B78002B00D0F6E00C2A42
:105CA00031D10F22A3789343E27812021343227971
:105CB000120413436279120613434B60E279A07910
:105CC00012020243207A00041043627A1206024351
:105CD000CA60E27AA07A1202024376484A8183427D
:105CE00008D804236E49142201980B7005F0BCFEFD
:105CF0001420C7E71201D21889235B059A42F0D815
:105D000001238B70BDE7022AFAD00523EAE76A4A2D
:105D100001239642E6D1FFF76BFA052F0CD9E37801
:105D2000A2781B021343227912041A4363791B06DB
:105D30001343624A0393136005F0E6FEA1E7584D52
:105D40002B78002B9DD1AB78002B00D1A0E02B89C4
:105D500001339BB20093B34200D091E0132AD4D90F
:105D6000CF7C8B7C3F02122120001F43FFF71AFFDC
:105D7000874200D08EE0002E3DD1E378A2781B024E
:105D800013432279E96812041A4363791B0613430B
:105D900003930A228B4212D1FF23A370E370237175
:105DA00063716B89002B09D1E37B227C1B021204F7
:105DB0001343A27B13431B0901336B8100226B89C0
:105DC000002B8ED0002A67D1686837013818000B85
:105DD0006B6900030390984205D9686105F064FD82
:105DE000EB780133EB7068681022A11C381805F0BD
:105DF00053FE2E8145E76F89009A7B1E9BB293422A
:105E00003AD1E278A37812021A43237905A81B0439
:105E1000134362796C6812061A43EB68009203928E
:105E2000211D0C22049305F01FFE0120260004A969
:105E300040421036FFF7E2FE013F012F17D1009AD2
:105E40000B232861824200D04CE704221C49200029
:105E500005F022FE042203A9686805F045FCE96804
:105E6000039AFF23914200D13CE7F73B3AE7310028
:105E7000FFF7C4FE1036DFE70923B742A4D831E7A5
:105E8000009BB34200D9FCE607232BE7022329E756
:105E9000032327E7062325E70A2323E7FFFE000065
:105EA0007443FF1F00000111FFFF000050485936E6
:105EB00001FF0000FFFF001102FF000034F000406E
:105EC0008043FF1F10B5034C0B000122210000F09E
:105ED0006BFA10BD856000110B8870B506000D00CF
:105EE0000224162B11D92B000322094900F05CFA79
:105EF000041E0AD1074B2A881B88191C934200D91B
:105F0000111C300089B200F0EFFA200070BDC046CD
:105F1000B16000113665FF1F10B54A780400013AE0
:105F20000B000220012A07D80A78002A04D0052293
:105F30002000024900F038FA10BDC046DF600011B1
:105F40000A7810B50B0004000220002A04D00722B2
:105F50002000024900F028FA10BDC0468B610011F4
:105F60000A7810B50B0004000220002A04D0092290
:105F70002000024900F018FA10BDC046F16100117E
:105F800010B5034C0B000B22210000F00DFA10BDE0
:105F90002162001110B5034C0B000D22210000F00E
:105FA00003FA10BD9362001110B5034C0B000F22D1
:105FB000210000F0F9F910BDED6200110A7810B56A
:105FC0000B0004000220002A04D011222000024904
:105FD00000F0EAF910BDC046FD620011002310B5C3
:105FE0001322190000F0E0F910BD000010B5034CB9
:105FF0000B001722210000F0D7F910BD4F630011EC
:10600000002310B51922190000F0CEF910BD0000D0
:1060100010B5034C0B001B22210000F0C5F910BD88
:1060200089630011F7B584890D0006000121002C59
:1060300022D000238268D3561778002B1EDA0C2C4E
:106040001AD90C3CA4B2131940880093230002F023
:1060500086FE431E984101307B06DB0F6B703F23A9
:10606000013C1F40A4B22870AF70AC80002C07D058
:10607000B3680133AB6000210800FEBD0020EBE7F0
:10608000AC60F8E70B7803704B8843704B881B0AB1
:1060900083700B79C370042070470420022B06D153
:1060A0000020537811781B02009A0B43138070472D
:1060B0000B8803700B881B0A437002207047042072
:1060C000009983420AD1537810781B0203430B8056
:1060D000D37890781B02034300204B807047F8B5BB
:1060E0000D004B7801240021461C03702B788B4255
:1060F00001D82000F8BD6B78B01C4F1C012B10D1CB
:10610000890069184B88022233704B88B9001B0A3A
:106110007370691805F070FA04360434A4B2F9B249
:10612000E4E7122359436B185A88043132705B88B4
:1061300010221B0A7370691805F05EFA12361234C9
:10614000ECE770B5049D14001E00052B01D8042057
:1061500070BD637812781B0213432B80E378A2781A
:106160001B02134302226B802A71211D681D063E0B
:1061700005F042FAB2B22A81E92AE8D82800A11D26
:106180000A3005F039FA0020E2E7002310B50A785A
:106190009A4201D8900010BD9A008A1854880133A1
:1061A00004705488DBB2240A447094888470928806
:1061B000120AC2700430EAE710B51100029C062BE7
:1061C00004D004201022142B01D010BD0222227111
:1061D0004B7808781B0203432380CB7888781B0216
:1061E000034363800431601D05F006FA0020ECE7EC
:1061F00010B50C788B7804315C43E4B20370220054
:10620000013005F0F9F9601C10BD0420022B06D105
:106210000020537811781B02009A0B4313807047BB
:1062200010B50C000A88023105F0E6F9208810BD8F
:1062300070B504000D0004981100012B01D8042052
:1062400070BD167852781202324302800200F13299
:1062500055701470E125002C00D10C35023B9AB228
:106260004280AA42EBD80231043005F0C5F9002083
:10627000E6E70420009983420AD1537810781B0284
:1062800003430B80D37890781B02034300204B809C
:10629000704710B50C000A88023105F0ADF920886E
:1062A00010BD000070B501211E000420049C0E40AA
:1062B0000B4218D1CB40DDB28D4214D90A49DBB272
:1062C000098899420FD32300EE331D703300580024
:1062D00011184978165C0902314301332152D9B2B1
:1062E0008D42F4D8002070BD8C43FF1F10B50C0008
:1062F0000A88023105F080F9208810BD10B50C78AD
:106300008B7804315C43E4B203702200013005F065
:1063100073F9601C10BD10B511000298032B01D851
:10632000042010BD14785278043B120222430280EC
:10633000CA788C781202224342809AB28280EB2A79
:10634000EED80431063005F057F90020E9E710B522
:106350000C000B8803700B881B0A43704B888370FA
:106360004B881B0AC3708A880430063105F044F953
:10637000A088043080B210BD0420012B03D100207E
:106380001378009A1370704710B50C000B880370D7
:106390000B881B0A43704A880230043105F02CF93F
:1063A0006088023080B210BDF0B589B003931E4BF7
:1063B000029242000700D05A019102F020F8132502
:1063C000061E2DD0029B01240370019B002B04D0DC
:1063D000001903999847001984B26B461B7A5BB287
:1063E000002B0FDA1021380002F01CFB19250028C1
:1063F00013D130003219E1B202F066FC051E0CD157
:106400000C34A4B2042304AA380005A9938006968C
:10641000948101F0AFFD051E02D0300005F0B4F903
:10642000280009B0F0BDC0463465FF1F70B50500F7
:106430000C0000280CD00020814209D0102220003E
:10644000044905F0D9F801202B7823736B78637326
:1064500070BDC046C0BD0011F0B506000D001700AC
:106460001C0085B002291BD00020102907D1022B67
:1064700007D0102B03D115E00020102C08D005B058
:10648000F0BD69463800FFF7D1FF2A0069460BE0EE
:1064900069463000FFF7CAFF22006946380004E071
:1064A000022BE9D12A003900300005F01DFBE6E798
:1064B000031CF02800D9F023032008499AB2013ABE
:1064C0000B80D317034006499B189B100B80D30FFA
:1064D00004499B185B100B807047C0469043FF1F18
:1064E0008E43FF1F8C43FF1F034B1B888B4202D33D
:1064F000024B4000C15270479043FF1F3465FF1F9D
:10650000014B4000185A70473465FF1F1722014B9A
:106510001A8070473465FF1F70B505000E2005F026
:1065200033FB041E13D0D023037000230622837094
:1065300007494570033005F05FF8064B2100DA8A01
:1065400062811B7E2373044B187805F055FB70BDE8
:106550005065FF1F4065FF1FE043FF1F262803D83B
:10656000024B4000C05A70470148FCE79243FF1FAE
:10657000FFFF000070B506000C00094D1C22002131
:10658000280005F069F8074B1E70074B1C7005F0DA
:106590005BFA0123002801D0002312202B7070BD6C
:1065A0004065FF1FE043FF1F6165FF1F70B50500D9
:1065B0000D4C0800E260A16010220021656005F02A
:1065C00083F8012803D11021A06802F058FD1022A1
:1065D0000021280005F078F8012803D11021606817
:1065E00002F04DFD70BDC0464065FF1F70B5041E32
:1065F00005D1002903D006220D4804F0FDFF0D4B04
:106600001D78012D11D1002C05D102221A7004F041
:10661000EBFF280070BD00221A70074B1B78FF2B80
:10662000F7D02000FFF778FFF3E70025F1E7C04639
:106630005065FF1F4065FF1FE043FF1F030010B5BB
:10664000002801D1002010BD00780B4A002803D19A
:106650005988D1821B7913761378022BF2D100234B
:10666000984200D103331370044B1B78FF2B01D0E9
:10667000FFF752FF0120E6E74065FF1FE043FF1FE1
:10668000002911D000280CD04B79012803D14022D9
:106690005242134303E03F221340032802D001205B
:1066A0004B7170474022F4E70800FAE770B5094DD6
:1066B0000100287800280BD0074C0622200004F0A7
:1066C0009BFF21002878FFF7DBFF200005F0E4F8AE
:1066D00070BDC0466065FF1F3A65FF1F00290AD0E4
:1066E000012808D13F224B799343C02B03D0403B74
:1066F0005A425341981C704770B5174D06002B78CD
:10670000FF2B15D00A2005F03FFA041E10D0D0232D
:106710000370C83B8370114B11491B784670C370DE
:106720000622043004F068FF2100287805F064FA9E
:106730000C4B1B78012B0DD10B4B1B68002B03D08E
:106740009B68002B00D09847084B04211878084A12
:1067500005F05AF870BDC046E043FF1F6065FF1F9B
:106760003A65FF1F5C65FF1F8865FF1F8C65FF1F73
:1067700060EA0000014B98687047C0464065FF1F03
:10678000014BDB68186870474065FF1F074B10B569
:10679000DA68136801331360054B1878FF2803D0BB
:1067A0008021C90105F018F810BDC0464065FF1FE3
:1067B000E043FF1FF7B50E0002F0C8F8051E1CD01D
:1067C0000E4B06621F78002F00D10778AB7910209E
:1067D000019305F0D9F9041E0FD0D0230380C73BE5
:1067E0008370019BE91DC3700622043004F004FF8E
:1067F00021003800E66005F0FFF9F7BDDE43FF1F1A
:10680000014B18787047C0466065FF1F054B002894
:1068100005D1054B1A78054B002A00D1014B180011
:106820007047C0465065FF1F6065FF1F3A65FF1F38
:10683000014B58687047C0464065FF1F024B1868FF
:10684000431E9841C0B270476465FF1F421E03009B
:106850000120152A03D9FF3B5A425341D8B2704751
:10686000F0B51C0000230E0085B0039002920B705F
:10687000029A934201D3002019E0E55C5A1CD2B27F
:10688000002DF8D0029851198142F4DC0233DFB2B6
:10689000A35C18000193FFF7D9FF002807D0013D42
:1068A000019A0399EBB233708A4202D1E01905B024
:1068B000F0BDDB19DBB2DBE710B50C0002F09EF88F
:1068C00003001220002B03D02100588804F08CFF15
:1068D00010BD000070B50E4D84006359002B15D01B
:1068E000186A002801D004F09FFE2B59586A00282E
:1068F00001D004F099FE2B59986A002801D004F0C9
:1069000093FE285904F090FE00232B5170BDC04621
:106910007065FF1F1C4B70B504000E0015009942F6
:106920000AD11A4B1B68002B01D1122070BD1B68C5
:10693000002BFAD09847F9E7154B994215D1134B24
:106940001B68002B0AD01B68002B07D09847002833
:1069500004D1104B1C70104B1D70E7E7290020007C
:10696000FFF7AAFF0028E1D1F3E7080001F0EEFFEE
:106970000028DAD003780320A342D7D129003000C1
:1069800004F032FFD2E7C046FEFF00006C65FF1F37
:10699000FFFF00006965FF1F6865FF1FF7B5040072
:1069A000808801F0D3FF0025A84203D00578A08895
:1069B00002F008F81C4E3378002B1FD0AB421DD1DB
:1069C0001A4B28001978FFF777FF002818D000230A
:1069D0003370A3790820A778A688019305F0D4F82E
:1069E000011E0DD0D0230370CA3B8370019B4770FA
:1069F00086808371280005F0FFF801E0002DE8D1C2
:106A0000A0880B4B8200D358002B01D0FFF762FF08
:106A10001721A088FFF768FDA08801F027FDA08856
:106A200001F0FEFDF7BDC0466965FF1F6865FF1FE9
:106A30007065FF1FF0B587B01D000CAB1B88070009
:106A400001930DAB1B88142002930EAB1B8816001C
:106A500003930FAB1B880091049310AB1B88059325
:106A600005F092F8041E1AD0D0230370CB3B477078
:106A70008370C670062229000430002D11D004F066
:106A8000BBFD019B21006381029B0098A381039BB6
:106A9000E381049B2382059BA37405F0ADF807B046
:106AA000F0BD04F0D9FDECE7F7B5009308AB1B8807
:106AB00007000C200D001600019305F065F8041E78
:106AC00013D0280001F042FF00280FD00078D02317
:106AD0002370C93BA370009B21002381019B677039
:106AE000A580E680638105F087F8F7BD014B187833
:106AF000EDE7C046E043FF1F13B504006489038936
:106B0000C2888188C0780094FFF7CEFF13BD0000D3
:106B100010B5044C2068002803D004F085FD002344
:106B2000236010BD7465FF1FA122F0B5818892001B
:106B30004A43384B384F1B6804009B189D22920033
:106B40009B18827989B01A603B68002B5FD01D7852
:106B5000324B1B68002B04D05B68002B01D0002057
:106B60009847260008363100E079FFF7B7FD237D0E
:106B7000E0710200E0780493638A29000393238A7A
:106B80000293E3890193A38800933300FFF752FF38
:106B9000E378002B0BD1E289A379A18802920196B8
:106BA000E27928000092012201F0DAFEE0703B68F1
:106BB000002B20D0FFF7ACFF194D287800281AD001
:106BC000184B1978FFF778FE002814D02B78E67858
:106BD00008200793A78804F0D7FF011E09D0D0230F
:106BE0000370CA3B4670837087808671079805F0F2
:106BF00003F800232B701721A088FFF775FCA088ED
:106C000001F034FCA08801F00BFD09B0F0BD064B8B
:106C10009DE7C0463409FF1F7465FF1F8865FF1F8D
:106C20006965FF1F6865FF1FE043FF1FF8B5070098
:106C300008000E0001F08AFE041E18D02620FFF77F
:106C40008DFC051E00D12578062004F09DFF041E52
:106C50000DD00021062204F0FFFCD0232370C23B9C
:106C600021006770A370A680E8B204F0C5FFF8BDEC
:106C7000F0B585B001930AAB1B78070002930BAB0C
:106C80001B7808000D000092039301F05FFE061EC2
:106C900022D0102004F078FF041E1DD01022002105
:106CA00004F0DAFC2620FFF759FC002800D13078E8
:106CB000D0232370C13BA370009B21002372019B52
:106CC00067706372029BA580A372039BC0B2E372DC
:106CD0000C9BE36004F090FF05B0F0BDF7B50D002C
:106CE000019001F033FE071E20D00E2004F04CFF6F
:106CF000041E1BD02620FFF731FC061E00D13E7873
:106D0000D0232380C53B0622A370F91DE01C04F0AC
:106D100073FC019B2A0063810123DD401A401D4062
:106D2000210022736573F0B204F066FFF7BD000026
:106D3000F0B585B0029010000D0017000A9E039375
:106D400001F004FE041E31D0029B002B2ED1039BC8
:106D500002795B0724D5122313430422002E08D1A5
:106D60000B99002905D10C99002902D10D99002910
:106D70001AD01A430D9B2271002B00D0C9E0002EBF
:106D800000D1CFE0002D00D0CCE0606A002801D017
:106D900004F04AFC1C21300004F0CEFC606205E0E7
:106DA00002239A430E33D7E793432371654BBA000E
:106DB000D458002C00D1AAE0002E10D0236A002B5A
:106DC00003D11C2004F068FC20625E4BBA00D3584B
:106DD000186A002803D01C22310004F00DFC0C9B23
:106DE000002B12D0574CBB001D596B6A002B03D1EE
:106DF000162004F051FC6862BB00E358586A002872
:106E000003D016220C9904F0F7FB0D9B002B11D038
:106E10004C4DBC006659B36A002B03D1142004F01A
:106E20003BFCB0622B59986A002803D014220D99BC
:106E300004F0E2FB380001F089FD051E67D0414BEC
:106E4000BA00D358002B62D01A6A3420002A00D12D
:106E50001C389A6A002A01D0143080B20B9A002A9A
:106E600001D01C3080B25B6A002B01D0163080B29A
:106E700004F08AFE041E4AD01822002104F0ECFB24
:106E80002620FFF76BFB0190002801D12B7801939E
:106E9000D0232370029B200063700A23294EA37025
:106EA000039BBD00A371AB59A780196A1830002954
:106EB00005D01C22A06004F09FFB200034307359E1
:106EC000996A002907D0030014221433E06002936A
:106ED00004F092FB02980B9B002B08D003001C22AD
:106EE0001C330B992061029304F086FB02987359BE
:106EF000596A002903D01622606104F07DFB6B46BD
:106F00002100187904F078FE3800FFF7E3FC05B0A3
:106F1000F0BD10220D9B0D991B69A018236204F08F
:106F20006BFB2CE70B9B002B00D13FE7012D00D022
:106F30003CE7606A002801D004F076FB1C210B9826
:106F40002AE7C0467065FF1F10B5044C2068002872
:106F500003D004F069FB0023236010BD6465FF1FAC
:106F60000B4B07B51A68002A01D100200EBD6946F7
:106F7000531C012012780731FFF772FC0028F4D06F
:106F800002780123100018401A42EED0EEE7C04606
:106F90008065FF1FF0B51F4F01203B6887B0002BB5
:106FA00025D09B78059300F0B3FB002821D00A2060
:106FB000FFF7D4FA04000B20FFF7D0FA164B0500B8
:106FC0001E78731E9E413B68F6B2191DD878FFF7F4
:106FD00057FB3B682900DA7A043303929A790193CC
:106FE0000292009033002000059A04F045FB07B0A0
:106FF000F0BDFFF7B5FF002805D00620FFF7AEFA79
:1070000004000720D8E70820FFF7A8FA04000920A9
:10701000D2E7C0466465FF1F6065FF1F70B50A4E6A
:10702000040033780D00FF2B0DD0042004F0ACFDDC
:10703000011E08D0D0230370CE3B45708370C4700E
:10704000307804F0D9FD70BDF043FF1F70B5040027
:1070500006200D0004F098FD011E0AD0D023037015
:10706000CD3B8370054B44701B688580187804F015
:10707000C3FD002C01D0FFF767FF70BD6465FF1FE3
:10708000F8B5264F06003B680D001124002B05D1F2
:107090000522234B1B78134202D112242000F8BD95
:1070A000204A10241268002AF8D01278002AF5D05D
:1070B000DB0719D52B789A1E012A1AD80C2004F068
:1070C000EBFA132438600028E8D000230A2243702A
:1070D00029000670023004F08FFAFFF75BFF041EF0
:1070E0000AD0FFF731FFD9E700F012FB0028E1D109
:1070F000E4E7002BE2D0D0E70B4B1B78032BCDD17C
:107100001D20FFF72BFA094B18800028C6D0084B2A
:1071100004211878074A04F077FBBFE76465FF1F76
:107120006165FF1F8065FF1F6065FF1F5E65FF1FB4
:107130008C65FF1F60EA0000F7B50193194B14003E
:107140001A78052306000F0012201A4221D00129C7
:1071500020D1154B1D68002D1BD002201F2C18D8E4
:10716000002C02D0019B002B13D0104B1F221E704D
:107170006E1C0021300004F06FFA019922003000EB
:1071800004F03AFA310020002C70002F06D004F0F1
:107190006BFAFEBD064B12201D68DCE704F00CFB09
:1071A000F7E7C0466165FF1F8065FF1FF043FF1FC3
:1071B0007C65FF1FF8B50F4E12243368002B17D0E3
:1071C0001B780F3C834213D100250B4F02213878E6
:1071D00004F0EAFC094B042138781D8004F0E4FC3B
:1071E000074B28001D8033685C7004F0C5FC040068
:1071F0002000F8BD6465FF1F8C65FF1F7865FF1FC9
:107200005E65FF1F70B5012823D11B4C2388002B1E
:1072100003D01A4A1578002D07D0194B1B68002B94
:1072200002D01878FFF7C6FF70BD3B2B02D93C3B5C
:107230002380F9E7134E0221307804F0B5FCFA22DE
:107240002388920002215A43307804F035FA2580D1
:10725000EAE70B4B1B68002BE6D00B4B1B785B0758
:10726000E2D5084B0221187804F09EFC0022024B64
:107270001A80FFF769FED7E77865FF1F5C65FF1F7F
:107280006465FF1F8C65FF1F6165FF1FF8B51E4D0C
:107290002868002803D004F0C7F900232B601B4E98
:1072A0003068002803D004F0BFF900233360184F82
:1072B00005243B7818002040234221D0154800F0D7
:1072C0002BFA3B78234213D0202004F0E5F9286004
:1072D000002813D02022002104F0BEF9202004F061
:1072E000DBF9041E306005D02022002104F0B4F93F
:1072F000002004E0286804F097F92C601320F8BD02
:1073000000F00AFAF4E7C0468065FF1F7C65FF1FA6
:107310006165FF1FE443FF1F10B50A4C23681A1E66
:107320000ED0002808D10130587004F025FC002848
:1073300005D02368002B02D00021FFF787FE012231
:10734000100010BD6465FF1FF7B5274E05003368B8
:107350000191181E21D05C78244F012C30D1FFF709
:10736000FFFD002825D02000FFF7F8F80400412891
:1073700014D91F4B022118781E4A04F045FA1E4BFF
:107380003C3C1C80022233685A703B78002B14D19D
:1073900028000199FFF75AFE0120FEBDFA22920053
:1073A0004243002AEED0124B0221187804F084F9EF
:1073B000E8E7FFF7D3F80200F3E700233B70EBE7C1
:1073C0003B78002BE8D1032004F0DEFB011E08D03F
:1073D000D0230370CC3B457083703368187804F079
:1073E0000BFCFFF7B1FDD7E76465FF1F5C65FF1F6E
:1073F0008C65FF1F60EA00007865FF1F10B5174914
:10740000838802008B4220D011D815498B4217D0B7
:10741000144900205B1899B2012907D892681178A5
:107420005A425341D8B2FFF7F9FD012010BD0E4A70
:1074300000209B1807229BB29A424041C0B2F5E758
:1074400083681878FFF768FFF0E7836899785A78BF
:10745000090218781143FFF777FFE7E70A200000D9
:1074600006200000F8DFFFFFAFDFFFFF014B1870C1
:107470007047C046F143FF1F10B5064C207001F065
:1074800041FA207804F068FB0521207800F062FDC5
:1074900010BDC0468C65FF1F0BB273B50D00002BED
:1074A00000DBC4E0884B187804F0A6FA041E0ED066
:1074B0000378912B0FD0A22B00D1A1E0834B187839
:1074C000FF2852D0210004F097FB00284DD18020E6
:1074D0000002684076BD43780F2B76D013D8052B79
:1074E00070D00E2BEAD18088794B98422BD8794BFB
:1074F00098421BD8784B9842E0D1A3681878591C61
:10750000FFF774F838E03E2BD8D18378032B74D082
:107510006CD8012B6ED0022BD0D1704B1B68002B86
:1075200023D05B68002B20D098471EE06C4BC0181E
:107530000C28C3D804F000FA1DC2C2150BC20B0BF5
:107540000B3223C23C00674BC0180728B6D8664BE5
:107550001B68002B09D01B68002B06D02000984721
:107560000AE0A3681878FFF7C7F8200004F064F871
:10757000ADE7A068FFF762F800289FD0F5E7A368A1
:107580001B78002BF1D0554B1B68002BEDD01B68EE
:10759000002BEAD0210055489847EDE74F4B1B6878
:1075A000002BE2D01B68002BDFD021005048F3E70E
:1075B000504B1B68002BD8D05B68002BD5D0210026
:1075C0004348E9E7FFF7EAF9CFE780884A4B98425A
:1075D00003D04A4B984200D070E7464B1B68002B03
:1075E000C3D05B68002BC0D02100D5E7153B012B31
:1075F000BBD963E7FFF798FAB7E7FFF77DFAB4E77F
:107600003F4B1B78042B07D100236A461380017976
:10761000408800F0C5FCA8E7364B1B68002BA4D0BF
:107620005B68002BA1D00100364898479DE70124F4
:1076300021420AD0294B1B68002B04D05B68002B29
:1076400001D000209847012043E78B070AD5264B3D
:107650001B68002B04D05B68002B01D020009847EA
:10766000022036E70421280008400D4200D131E70E
:10767000254E3388002B21D0013B9BB23380002B59
:107680001AD1FFF7DBF800280AD0204B1C70164BEC
:107690001B68002B04D05B68002B01D020009847AA
:1076A000FFF7C6F8694601F001FD6846FEF7FEFFE8
:1076B0001D20FEF753FF308004200AE7024B1878A4
:1076C00004F072FAF8E7C0468C65FF1FF143FF1F14
:1076D0000E20000001200000091000008465FF1F3B
:1076E000FEDFFFFFAFDFFFFF8865FF1F0C200000FC
:1076F0000B2000006C65FF1F0D2000001320000010
:107700006165FF1FFFFF00005E65FF1F5C65FF1FD7
:1077100010B501F09BF910BD014B18607047C046D1
:107720008865FF1F0B880020162B01D81723042023
:10773000014A13807047C0463665FF1F002070471E
:10774000074A03001188814207D09188002099429E
:1077500002D101308000101870470020FAE7C046BF
:107760009465FF1FF0B58F7806000D00C5B01E2F81
:1077700015D1FFF7E5FF051E03D10024200045B019
:10778000F0BD00223B003100C078009200F0B2FB57
:107790000400A81C00F0D2FBFF23EB70EEE7264BA1
:1077A000062403931B78FF2BE8D0182FE6D87B081C
:1077B000224A013BDB0002929A589446002ADDD00F
:1077C000029AD3185B68002BD8D00878002802D121
:1077D0004B78012B02D10624122FCFD107AFAB88F3
:1077E000697800976446AA68A047041EC6D1AB78A2
:1077F000029A5B08013BDB00D318390030005B685C
:107800009847041E0BD1AB78042BB6D0039A3100F5
:1078100010782200009700F06DFB0400AEE76A7854
:10782000002AABD1AA7805A93B88087130000A70FC
:107830004B80FEF747FBA0E7F443FF1FD0BD0011CC
:107840001D4B37B5050098420BD000290AD1FFF730
:1078500077FF002805D11948FFF772FF002800D0F4
:10786000058037BD01291AD1FFF76AFF041EF8D041
:1078700001235B420380A378FF2BF2D0FE2B07D0BD
:107880000023E0781422009329001E3300F032FB1D
:10789000A01C00F053FB01235B426380E1E7022957
:1078A000DFD1013901F0BEF80028DAD12800FFF756
:1078B00047FF041EDFD1D4E7FEFF0000FFFF0000FA
:1078C000022210B5074B52421A80074801325A80F3
:1078D0009A80DA8000F07EFA044801F025F8002052
:1078E00010BDC0469465FF1F6577001141780011F7
:1078F0000388F7B50400002B02D102252800FEBD45
:1079000042680221137825485268FEF7A5FD002839
:107910002ED0234F01253A88002AEFD080232188DA
:107920005B0201259B1A9942E8DC0C2003F0B4FEAF
:10793000061E31D03B8822889C4600231800019502
:1079400061469DB2491989B2AA421BD8002801D0CC
:1079500062443A8000233000082208C0210003F06E
:107960004BFE104A1368002B13D100251660C5E7A3
:107970006268022113780C485268FEF76DFD0028FA
:10798000C7D1BAE760681D014019418101330198F0
:10799000D6E71A001B68E6E71325AFE73EBE0011E5
:1079A000F243FF1F9065FF1F3CBE0011014B187092
:1079B0007047C046F443FF1F14230A0010B51A4055
:1079C000194204D00122102101F048F810BD4B06E5
:1079D000F9D4012088434000F8E710B514008B0665
:1079E00004D50122102101F039F810BD08230A0046
:1079F0001A40194202D14BB2002B0FDA102101F0CC
:107A00002DF8002808D02300F2331B78002BECD08F
:107A1000F1342378012BE8D10020E6E70320890721
:107A2000FAD4E2E7F0B51F00184B85B01C6801904E
:107A300002910392002C27D1200005B0F0BDA5686B
:107A40003301ED186B89019A934211D3029A934244
:107A50000ED8002F04D10A9B002B10D12C00EBE78D
:107A60003B002978039A6868FEF7F6FC0028F2D1FB
:107A70000136B6B2A388B342E1D82468DAE7A36836
:107A80000A9A5B891380E9E70026F3E79065FF1FF8
:107A900037B50C000A8849880123914217D3002A80
:107AA00015D0651D23792A0002210A48FEF7D4FC6F
:107AB000102300280BD023796188208800242A0015
:107AC0000094FFF7AFFF0A23A04200D02300180064
:107AD0003EBDC0463EBE001113B50A000888498865
:107AE000012388420BD8002809D0002413790532DD
:107AF0000094FFF797FF0A23A04200D0230018004C
:107B000016BD13B50A0008884988012388420BD89E
:107B1000002809D00024137905320094FFF782FF72
:107B20000A23A04200D02300180016BDF0B58BB088
:107B300003904A8808880E000123824255D300280A
:107B400053D00023012704AC237000227188130056
:107B50000092FFF767FF051E3ED02078002835D140
:107B60002B78022B18D167706A8983000130E318E3
:107B700080005A8069680222201803F03DFD2378B6
:107B80000133DBB22370042B19D93B006889013023
:107B900080B2002BD9D01FE0022363701223584318
:107BA0006A89231804305A8069681022201803F06B
:107BB00023FD23780133DBB22370002BE5D10C4A7F
:107BC0006B899B185A425341DBB2DFE76378012B84
:107BD000E4D12B78022BC7D022780A23002A04D0C4
:107BE00021000398FEF798F9002318000BB0F0BDB0
:107BF0000100FFFF0F4BF0B504001868002816D0F5
:107C000083685D89A54207D88288AE18B44203DA3A
:107C100012019A18934201D10068EFE71E005F89B4
:107C20001036A74204D1002900D00D801800F0BD05
:107C30003300EFE79065FF1F70B505000C00088862
:107C40000021FFF7D7FF03000120002B04D0220002
:107C50002800197AFFF7C1FE70BDF7B50C000025AA
:107C600001902300EE331B78AB4201D800200AE0DC
:107C70006B00E65A00213000E718FFF7BBFF002831
:107C800002D126800130FEBD017A0198FFF794FEF3
:107C9000002802D03B882380F5E70135EDB2E0E70C
:107CA00010B5040008880021FFF7A4FF030001209D
:107CB000002B03D02000197AFFF77EFE10BD0000D4
:107CC000054B1B68002B01D1180004E09A6852890B
:107CD0008242F6D1988870479065FF1FF0B50E2755
:107CE000002687B0039302ABFF183E8005001F4BB0
:107CF00040891400984207D02B78013000976A68B9
:107D000080B2FFF78FFE060002212B7818486A68C0
:107D1000FEF7A2FB00280FD06C892000FFF7D0FFF0
:107D2000002802D0013C0419A4B2039B002B00D010
:107D30001C80300007B0F0BD02212B780D486A6826
:107D4000FEF78AFB0028E7D102212B780A486A68EF
:107D5000FEF782FB002807D0002EDED03B88A3422E
:107D6000DBD17489013CDFE76C89DEE7FFFF0000AF
:107D70003EBE00113CBE00113ABE001110B50C0011
:107D8000FFF7DEFC03000220002B0AD0002C00D0FD
:107D900023609B781720FE2B03D00138FF2B00D1E6
:107DA000002010BD73B50D0001A904001600FFF7F7
:107DB000E5FF172805D0002E04D129002000FEF78A
:107DC00027F976BD01221021200000F047FE00288F
:107DD000F3D0F6E7014B18607047C046A065FF1F5F
:107DE00037B56B469D1D010004000222280003F0F8
:107DF0003BFE2B88B02B0ED12379122B09D1230007
:107E0000FA331B78012B06D10121608800F0E0F8DD
:107E100001E01B2BF8D037BD10B5054B04211870BD
:107E200000F098F8FFF74CFDFEF770FB10BDC04660
:107E3000A465FF1F0020F0B50BB20F0087B083428E
:107E400034DA274B187803F0D7FD051E2BD00378C2
:107E5000A02B25D103AE3100FEF7E4F8041E0BD1B0
:107E6000B378DB0724D51F4B06341B68002B03D0E7
:107E70003100688898470400A868002801D003F002
:107E800083FC002C08D1184A039B1340174A9342E5
:107E900006D0B3781B2B03D00121688800F098F836
:107EA000280003F0C9FB80200002784007B0F0BD35
:107EB0000F4B1B68002B10D0310068889847041EB8
:107EC000DAD07378002BD7D1B27801A90A704B8031
:107ED0000C716888FDF7F6FFCEE70624F1E7C0468F
:107EE000A465FF1F9C65FF1F00FFFF00000112003B
:107EF000A065FF1FF7B50190FC200D0017001E00C4
:107F000003F042FE04001320002C12D0B023200006
:107F10002370089BF4226770658026710830002B5F
:107F200008D0190003F068FB2100019803F064FEFB
:107F30000020FEBD089903F08FFBF5E710B5041E85
:107F400006D00078FD2803D803F02EFCFF23237011
:107F500010BD00000A1F93B210B504000220032BCD
:107F600005D882400020024BD1529B189C7010BD56
:107F7000C465FF1F0B8870B5043B04000D00022090
:107F8000032B0BD80121200000F04CFD030014202E
:107F9000002B03D02900200000F0DEFB70BD0000A4
:107FA00007B51300034A00920A00012100F02CFCDF
:107FB0000EBDC046DD81001107B50192032200927B
:107FC000024B0A00122100F049FC0EBD5B82001139
:107FD00007B56B4601AA11800449D880087806339A
:107FE000012802D1190003F087FB07BDA565FF1F1B
:107FF0000C4B10B518700023FF210B4A138013811E
:1080000093819380094A53801370517293819372C4
:10801000D174D3821375517703F076FC00F0FCF92C
:1080200010BDC046D465FF1FC465FF1FA665FF1FB6
:10803000F0B58DB06B46002003910C229B5E83420D
:1080400000DBB0E05D4B187803F0D6FC051E00D1D4
:10805000A4E00378902B00D09DE006AF0100468895
:10806000380000F013FA79680400002900D19CE080
:108070003B88052B6ED13B89032B1CD905AC200016
:1080800000F0A2F86288172A61D83989131D994235
:1080900031D17968237804310291D90738D56078D5
:1080A00000F08EF9071E06D0002303712378012B00
:1080B00008D0132B23D0A868002800D178E003F063
:1080C00063FB75E06288029909A800F0A6F80290A7
:1080D000380000F08BF909AA2378387A019200223F
:1080E00031000092029A00F012F9380000F064F9B1
:1080F000029B002BDFD0300000F080F9DBE7037833
:10810000032BD8D16288029909A800F0D6F8DEE7DF
:10811000122B13D1029909A800F0B5F8021EEAD17A
:1081200027498B88002BC6D0887909A9237801912B
:1081300061780091310000F0EAF8BCE7002302AA60
:1081400093833000617809AAFFF72AFFB3E71D4B3C
:108150000993F6E7042B02D09A1F012AABD8184ADC
:10816000043B9B00995A0029A5D0D2189078310081
:108170003A0000F0AEF800289DD13B88042B03D0D4
:1081800001213000FFF724FF012C04D1A86800284A
:1081900001D003F0F9FA280003F04EFA8020039B87
:1081A0000002434018000DB0F0BD012800D182E765
:1081B00001213000FFF70CFFEDE7C046D465FF1F3B
:1081C000C465FF1F010017000B7803704B784370E4
:1081D000CB788A781B021343438070470A880300D8
:1081E00002700A88120A42700A88012A06D14A8857
:1081F00082704A88120AC2700420704702208242AC
:10820000FBD14A8804309A704A88120ADA708A8848
:108210001A718A88120A5A71EFE710B5040001201A
:1082200082420CD94B780A781B0213432380834285
:1082300006D1CB788A781B0213436380002010BDDF
:10824000022BFBD1CB788A781B02134363804B79D6
:108250000A791B021343A380F0E70B8803700B8895
:108260001B0A43704B8883704B881B0AC3708B8832
:1082700003718B881B0A4371CB888371CB881B0ADF
:10828000C3710820704703000120082A14D14A78DE
:108290000878120202431A80CA78887812020243D0
:1082A0005A804A790879120202439A80CA798879F9
:1082B000120202430020DA80704710B5040001204A
:1082C000022A05D100204B780A781B021343238031
:1082D00010BDF8B5060010200F00150003F054FC87
:1082E00004000120002C0ED0A0230C2229002380A2
:1082F0006780201D002D07D003F07EF9210030009B
:1083000003F07AFC0020F8BD03F0A6F9F6E7F7B514
:108310001E00009008AB142017001D78019103F097
:1083200033FC041E12D0A2230370019B47704380CC
:10833000099B057146710C220830002B07D01900EB
:1083400003F05AF92100009803F056FCF7BD099993
:1083500003F082F9F6E737B5041E0FD04388002BEF
:108360000CD00025C1881323007A172201950095AF
:10837000FFF7CDFFFF2365806372257037BD0000D6
:1083800010B50C4904004A88002A09D08B89002BBB
:1083900005D00020CB8A0222834201D010BD0122E9
:1083A00013000A20434300204032C854C8184280BA
:1083B0000472F3E7A665FF1F002343800370704734
:1083C000094B00211A0010B55C88002C06D01C79DE
:1083D000844203D10A234B43D01810BD01310A3324
:1083E0000329F1D10020F8E7A665FF1F10B50400AE
:1083F000407A03F0D9F9FF23637210BD704704304F
:1084000010B580B203F0A0FA002803D0042149423D
:1084100003F0C2FB10BD000070B50025104CA06831
:108420002580A581A580A84202D003F0ADF9A56002
:1084300000250C4C0C4B606D1D80230058331D70C3
:10844000A84202D003F0A0F9656500256068002805
:1084500001D003F099F9013508340A2DF6D170BD29
:108460006C66FF1F1066FF1F6066FF1F70B5041E5D
:1084700009D1054D2880A881A880A868002802D0CD
:1084800003F082F9AC6070BD6C66FF1FF0B54B88DD
:1084900085B00193002343600A7905000F00022A8A
:1084A00000D07BE0CA88032A17D98B685E781978D8
:1084B0003602DC78D8790E4399781B7A24021B02A5
:1084C0000C43034353495BBA0B80331D93421ED1C7
:1084D000042C04D0631F022B0ED9012015E0019A51
:1084E0004D4B1201D35A002B06D00198FFF7BEFF67
:1084F0004A4A1369013313610421B8682E812C8024
:10850000494203F049FB6860002005B0F0BD434DCF
:10851000042C06D0631F022B0FD9EB680133EB60EC
:10852000DBE7019A3C4B1201D35A002B05D001988E
:10853000FFF79CFF2B6901332B61374B300002930F
:10854000019B029A1B010193002301998C468B52D7
:10855000130063449C8003939E81FFF750FF039BAD
:10856000041E986016D00421B868494203F014FB39
:10857000FA880100043A200003F03EF80199029ABB
:10858000FB888A5A043B9B18029A8B522B68013352
:108590002B60A2E7AB690133AB619EE71E4B0293F0
:1085A000019B1E01029BF35A002B2DD002998C19BE
:1085B000A068002828D0012A26D1FA889B189BB2EF
:1085C0007352A189994217D39B1AC018B96803F056
:1085D00013F8029BA289F35A934200D07DE7002250
:1085E0002B81A3882B80A3686B60029BF2520B4AFD
:1085F00053680133536070E7084A9368013393600E
:108600000198FFF733FF68E7044A53690133536168
:10861000F6E7C046D665FF1F6C66FF1FDC65FF1FCF
:1086200070B5051E15D10B4C0B4B18802300583329
:108630001870606D002802D003F0A6F8656525006B
:1086400050356068002801D003F09EF80834AC4231
:10865000F7D170BD1066FF1F6066FF1FF0B51700F1
:10866000A12285B0920001934243394B06001B685A
:108670000C009B18D933FF331D78FDF741FF043000
:10868000854204DD3000FDF73BFF0430C5B2BD423A
:1086900007D33A0000213000019B02F0F5FF05B03E
:1086A000F0BD2900380003F0CFF82300C6B25033E4
:1086B0001E700393019B29006365380003F084FA60
:1086C000CBB20293002B02D0039B01361E70002612
:1086D0002300503303931B78B34204D8606D002805
:1086E00031D10020DBE7029A2800002A04D0013BA8
:1086F0001000B34200D02800F700E719387003F0EB
:108700002BF8786000280ED03A78019902F074FFB7
:10871000019A3B780136D3180E4A0193D369F6B219
:108720000133D361D4E7039B18706065A74205D17C
:10873000084A1320D36A0133D362B0E7606803F0BC
:1087400023F80834F2E703F01FF800236365C8E755
:108750003409FF1FDC65FF1FF7B50D00070004217A
:10876000686803F019FA2B89040003702B891B0A2F
:1087700043702B8883702B881B0AC3702E890225B7
:108780000436F6B2F42E15D81B4B9F4214D10C20A0
:1087900003F0FAF91135011E0CD0902303708E3BC3
:1087A0000371043B4380154B8460C680187803F046
:1087B00023FA00252800FEBD5C237B43104AD31812
:1087C0000093583301931B78002B0FD10300320024
:1087D00038000099FFF742FF019B05001B78002B32
:1087E000E8D13800009902F0C7FFE3E7054A072502
:1087F000536A01335362DDE7FEFF0000D465FF1FBB
:108800001066FF1FDC65FF1FF0B587B000901720D2
:108810000F0016000193FFF7F2FD1325041E19D077
:108820000C98031E02D00199201D9847030AE3709B
:10883000052302AAA070043090812770009866700A
:1088400003A993800494FFF787FF051E02D0200040
:1088500002F09AFF280007B0F0BD0000F0B587B025
:108860001F000CAB1B780391059301210DAB060093
:108870001C78049200F0D6F81425002821D020009E
:10888000FFF77EFD0135041E1BD01149059B0A78B8
:1088900003700132D2B2131EC68001D101231A0027
:1088A0000B7022713000049B03990097FFF7ACFF17
:1088B000051E09D1230021000648074A093303F0A9
:1088C000BBF8280007B0F0BD002363802370F8E7F1
:1088D000D865FF1F5783001130750000F8B50500FB
:1088E0000E00064C064F2368002B02D031002800F2
:1088F00098470434BC42F6D1F8BDC0467C66FF1FE1
:108900009066FF1F0123064A5B42538000231371C8
:108910005362044A136053609360D36013617047DD
:108920009066FF1F7C66FF1F0200002310B50649FA
:108930009C000859002801D1625010BD0133052B5D
:10894000F6D11320F9E7C0467C66FF1F034A53881F
:10895000181A434258414042104070479066FF1F2A
:10896000F0B585B002930AAB1F780CAB1B88009062
:1089700008000E0001920393FFF7E8FF05001120A5
:10898000002D1BD10E48FFF7E1FF04001520002C3D
:1089900014D006220B99A771E01D02F02DFE019B59
:1089A00030002371029B29006371009B6680237055
:1089B000039B6562E381FFF791FF280005B0F0BDDE
:1089C000FFFF000010B5FFF7C1FF04000220002CDC
:1089D00012D060880121FFF781FF606A002801D072
:1089E00002F022FE28220021200002F035FE0123A1
:1089F00000205B426380207110BD000030B5074A43
:108A0000074C5588010013780020A54204D05B1A5A
:108A100059424B415842104030BDC0469066FF1F3E
:108A2000FFFF0000084A10B501230C00904208D057
:108A3000FFF78CFF031E04D0037923405A1E934195
:108A4000DBB2180010BDC046FEFF0000024B1879D3
:108A5000431E9841C0B270479066FF1F70B5040076
:108A60000D001600FFF772FF002804D10D4B9C4249
:108A700000D0143070BD416A03790520002907D069
:108A800012221A40102A02D10520002EF2D10F2006
:108A9000DB06EFD5897E0C20A94289414942494233
:108AA0000840E7E7FEFF0000030010B5002800D1F2
:108AB00010BD0348034A41889142F9D09847F7E72F
:108AC0009066FF1FFFFF0000002330B5C45CCD5C43
:108AD0006C40D4540133102BF8D130BD0F23002249
:108AE00010B5C45C64002243CA54C25CD209013B85
:108AF000F7D210BD0200010010B52032103102F093
:108B00006BFD10BDF0B58BB00390102005931700DE
:108B1000049102F0C1FD0090102002F0BDFD009B09
:108B200013240190002B05D000280CD113240098A9
:108B300002F07AFD019B002B02D0180002F074FDB8
:108B400020000BB0F0BD102002F0A6FD06001020A2
:108B500002F0A2FD13240500002E00D1AEE0002893
:108B600019D01022002102F077FD3200290003986D
:108B700002F032FD041E0ED133787F2B51D8300025
:108B80000099FFF7ABFF009B1B787F2B53D801990F
:108B90000098FFF7A3FF300002F046FD002D02D041
:108BA000280002F041FD002CC1D1102002F074FD1C
:108BB0000600102002F070FD0290002E7CD00028EC
:108BC00078D03A000F3223000125121105D00F335F
:108BD0003B4015B25A4253411BB26A1E1201002B90
:108BE00033D0049BD2B298180099029AFFF76CFF19
:108BF000013D10220021300002F02EFDADB2049F95
:108C00002D017D19AF4242D0002C33D0300002F04C
:108C10000BFD029B002B00D189E7180002F004FD38
:108C200085E729003000FFF759FF28002549009A01
:108C3000FFF74AFFA7E729000098FFF74FFF28003A
:108C40002049019AFFF740FFA5E70F210F40049943
:108C50008A18D9B28F4208D9D15C06A819540133B9
:108C6000102BF6D1029A0199C0E7791A4842414186
:108C7000C901F2E73900300006AAFFF725FF3200EC
:108C8000039806A902F0A8FC10370400BAE7002CEC
:108C9000BCD13000029906AAFFF716FF320006A9E0
:108CA000039802F099FC082204003100059802F0B4
:108CB000A3FCABE71324A9E71324AAE7002800D0FC
:108CC0006EE733E744BE0011F0B58BB00F0016001D
:108CD0000225009000283FD0002A3DD00B1DDBB2BA
:108CE0001800029302F0D8FC1135041E34D0FDF7B1
:108CF00047FD05003A000099201D02F0A5FCEBB2EB
:108D00000393E3702B0CDBB22F0A00936370FFB266
:108D10002B0E2370A7700193FDF72CFD102201008C
:108D200006A802F091FC2100029A04AB06A8FFF706
:108D3000E9FE051E0DD1039B08223370009B04A998
:108D4000B370019B7770F370301D02F07DFCFDF76E
:108D50001DFD200002F068FC28000BB0F0BDF0B54E
:108D60008FB00D00149E039004920593002A03D146
:108D7000022420000FB0F0BD002EF9D00398FFF7B9
:108D8000E5FD1424071EF4D07278337812021A43DA
:108D9000B3781B041343F27812061A43036A019254
:108DA000934201D30133E3D1002D03D03B79012459
:108DB0009B07DED50822002106A802F04DFC059B8A
:108DC00013240433DBB21800029302F065FC051E85
:108DD000CFD0059A0499043002F036FC0422310009
:108DE000280002F031FC3900102210310AA802F0EC
:108DF0002BFC2900029A06AB0AA8FFF783FE041E8B
:108E00000FD1082206A908A802F01EFC0822311D75
:108E100008A802F069FE012807D101990398FDF71F
:108E2000C9FC280002F000FCA3E70124F9E70000D8
:108E300070B51C4C05002368181E10D0002D14D1ED
:108E40001A78002A0CD1981C083202F0D5FB02F0E7
:108E5000D3FC0135002808D123681D70012070BDA6
:108E60000A331800082202F0C7FB2368002BF5D054
:108E7000122002F089FE061E0DD0C1232168037066
:108E8000457002311022023002F0B6FB2368310037
:108E9000587802F0B1FE206802F0C6FB0023236080
:108EA000DCE7C046B866FF1FF8B504002020FDF7D8
:108EB00055FB0D4EA700BB590500002B0DD0002817
:108EC0000BD0D878FF2809D108492A000C55F3594E
:108ED00007480333611802F0AFFDF8BD290002F026
:108EE000C3FC0028F0D1F8E7D466FF1FBC66FF1F63
:108EF00001A1001170B5064D84006359002B05D007
:108F0000D87802F051FCFF226359DA7070BDC04678
:108F1000D466FF1F70B506008CB00C001500002150
:108F20003022684602F098FB31001022684602F0B9
:108F30008BFB1D2021000322684402F085FB68465C
:108F4000FFF7D8FD2D21040003222800694402F018
:108F50007BFB20000CB070BDF0B50700160097B089
:108F600001931CAB1D7830221EAB00910AA8002192
:108F70001C7802F071FB102239000AA802F064FB91
:108F80001022002102A802F067FB0722310002A88C
:108F900002F05AFB072202AB9818631E9C4101990C
:108FA00002F052FB02AB9C732B005A1E934102AAA3
:108FB000D3730021102206A802F04EFB06221D9951
:108FC00007A802F041FB1A2002ABC01806221F9925
:108FD00002F03AFB102200990EA802F035FB102295
:108FE00002AB0EA908781C78013A6040D2B2087032
:108FF00001330131002AF5D10AA8FFF77BFD1022C9
:1090000012A904000EA802F0F7FA102206AB0EA96E
:1090100008781D78013A6840D2B2087001330131F6
:10902000002AF5D10AA8FFF765FD04431022209815
:10903000E4B212A902F008FB200017B0F0BD70B531
:109040000E0014008CB00100102268461D0002F0D2
:10905000FBFA3100082204A802F0F6FA21000822E7
:1090600006A802F0F1FA6846FFF744FD040010225A
:10907000280008A902F0E8FA20000CB070BDF8B58D
:1090800006000D0000243719AC4200D3F8BD02F0F1
:109090009BFC030A3B70631CDBB201379D4203D982
:1090A0000234F054E4B2EEE71C00EDE773B50600BD
:1090B0000C000225002819D0002917D0032101A88F
:1090C000FFF7DDFF6B469A793F231A4001331343C4
:1090D0006A463000937101A92200FFF71BFF051EAD
:1090E00004D10322E01C01A902F086FA280076BD13
:1090F00003785807DA08C00FD20080009B0710439E
:109100009B0F1843C0B2704707230B40C908C90022
:109110000B4303707047000070B50400FFF7EAFED0
:10912000134DA4006359002B21D0186A002801D0E8
:1091300002F07AFA2B59986E002801D002F074FAE6
:109140002B59D86E002801D002F06EFA2B59186FF7
:10915000002801D002F068FA2B59586F002801D07E
:1091600002F062FA285902F05FFA00232B5170BD19
:10917000D466FF1F0E4B8000C35870B50C00002B47
:109180000FD09D68002D0CD02B78201D0B706B78B4
:109190004B70A97CFFF7B8FF2B7E23726B69E360ED
:1091A00070BD10220021200002F056FAF8E7C046F8
:1091B000D466FF1F014B18607047C046D066FF1F82
:1091C000074A03008000825810B5002A06D0D088D4
:1091D000984203D1012901D1FFF79EFF10BDC0467F
:1091E000D466FF1FF0B5264E95B087000B93BB5990
:1091F0000500099112200A92002B31D0D888FFF780
:10920000A5FB04001420002C2AD0280010A9FFF789
:10921000B1FFBB591E781D6A002E23D00895FDF7BB
:10922000EFFA07000020FDF7F1FA0790A379E61D99
:10923000069310AD0CA9089800F0E2FA0EA92800D8
:1092400000F0D7FA0B9B0A990493069B09980293A6
:10925000079B0396019300970EAB0CAAFFF77CFEC9
:1092600015B0F0BDFDF7CCFA06903000FDF7CEFA50
:10927000E31DA779079310AB06000893DAE7C04611
:10928000D466FF1F30B50C4C85002A59030085B009
:109290000120002A0ED018006946FFF76BFF2B59FA
:1092A0001A78D888054B002A00D1054B6A46072159
:1092B00000F0D9FB05B030BDD466FF1FF397001155
:1092C0000198001130B5094C8500295985B010224C
:1092D0006846253102F090F92A591121044BD088B3
:1092E0006A4600F0C0FB05B030BDC046D466FF1F23
:1092F0009D98001130B5094C8500295985B0102280
:109300006846353102F078F92A591121044BD0888A
:109310006A4600F0A8FB05B030BDC046D466FF1F0A
:10932000DB980011F7B54D4F86001020F4590D0061
:1093300002F0B2F9F3592062186A132200286CD0A7
:10934000033A29009C6802F057F9F3591A78019200
:10935000002A58D11E6A227D317B94465140012259
:10936000019F114201D167461740217D9143394346
:109370002175377B4F40BC4660460027800701D4EB
:109380004F081740012102208F40227D82433A433B
:109390002275377B5740BC4660460027400701D402
:1093A00097080F400420227DBF0082433A43227574
:1093B000627D002794466046727B42400A4201D19A
:1093C00067460F400121627D8A433A436275777B8D
:1093D0005740BC4660460027800701D457080F401D
:1093E0000220627D7F00824317436775767B0022EF
:1093F0007E40760701D4BA080A400426617D9200B7
:10940000B1430A4362756A78002A08D06278002A5C
:1094100005D005220533DA7700221000FEBD0422B4
:109420002979114205D1A17C114202D10533033AB9
:10943000F1E7019A21782C78002A02D10A00210054
:10944000140018220429E8D8042CE6D8052060432B
:10945000034A05331218525CDDE7C046D466FF1F8D
:1094600054BE001110B50A001121024B00F0FBFAA6
:1094700010BDC046379900110B0030B587B001AD63
:109480002B806B4604001100981D082202F0B4F8EE
:109490002A000B212000024B00F0E5FA07B030BD96
:1094A0005F99001110B50A001121024B00F0DBFAA0
:1094B00010BDC046B399001113B50B0011006A46E8
:1094C00013706B4604000622581C02F095F86A4699
:1094D00008212000014B00F0C6FA13BDD3990011FA
:1094E00010B50A001121024B00F0BDFA10BDC046B4
:1094F000239A00117FB505000B4BAA00D458080031
:10950000002C0FD0666F237FE28821780396266FA8
:109510000296E66E0196A46E0094FDF709FC280001
:10952000FFF7FAFD7FBDC046D466FF1F10B51721B7
:10953000FFF7E0FF10BD000070B50A000D00064BFC
:109540000221040000F08FFA060029782000FFF7BE
:10955000D1FF300070BDC0460399001170B586B0D0
:1095600000236A461370836804001D78681E0A2869
:1095700059D801A902F0F8FA060633373B3F4347B2
:109580004B4F5300180000F042F9062312284BD02D
:1095900000281BD16088FFF7D9F90823002813D0D1
:1095A0004279002A47D1264B1A78072312070BD598
:1095B000244B1A680723002A06D01668002E03D011
:1095C000290001AAB04703006A4613706B461B7856
:1095D0006088002B2AD1FFF767FC06B070BD180029
:1095E00000F06CF9D4E7180000F087F9D0E7180014
:1095F00000F093F9CCE7180000F0ADF9C8E71800C7
:1096000000F0C3F9C4E7180000F0F6F9C0E718004D
:1096100000F0F6F9BCE7180000F013FAB8E71800FC
:1096200000F013FAB4E707236A46137069466088AE
:10963000FFF782FFD1E70523012AC5D1024BB8E726
:109640006165FF1FCC66FF1FD066FF1FF8B52C4F6A
:109650008600F35904000D00002B40D0DA888242C6
:109660003DD15A78062A33D11A78002A2ED001200B
:1096700099681A6A097D014206D0157B054203D01C
:1096800007225A700120F8BD0220014204D0157B48
:10969000054201D00922F4E70420014204D0127BE4
:1096A000024201D00B22ECE7164B1B68002BE9D0DD
:1096B0005B68002BE6D020009847BB5900215B78FF
:1096C000122BDFD12000FFF715FFDBE70E4BECE795
:1096D000112A04D1002900D032252900F2E7002DFB
:1096E00008D12000FFF732F9002803D010230279B7
:1096F0001343037121002800FDF798FAC2E7C04622
:10970000D466FF1FCC66FF1FD066FF1F70B50E4EDC
:109710008500AB590400002B13D01B78002B11D10E
:109720000A4B1B68002B04D05B68002B01D0200083
:10973000984773595B78122B03D100212000FFF763
:10974000D9FE70BD024BECE7D466FF1FD066FF1F49
:10975000CC66FF1F094B8000C3581020002B0CD093
:109760001A6A002A09D09B68002B06D0127A1B7E49
:10977000101C9A4200D9181CC0B27047D466FF1F53
:1097800070B503000D0014000220002A30D000291B
:109790002ED013700B78081D53704B789370FFF721
:1097A000A7FCE070012002212B7A23716B7B034020
:1097B00063716A7B0A401343042263716E7B164017
:1097C000334363716E7BF608F600334363712B7B82
:1097D0000340A371287B014000200B43A371297B28
:1097E0000A401343A3712A7BD208D2001343A3710A
:1097F00070BD10B50A0001000120FFF7C1FF10BDC8
:1098000010B50A0001000220FFF7BAFF10BD70B5C5
:1098100006000C000220002E30D000292ED07378D4
:10982000201D0B70B3784B70F178FFF76DFC0122AF
:109830003579257271794B10080013409340104020
:109840000343881010408000C9080343C9000B433C
:109850006373B1794B1008001340934010400343E9
:10986000881002409200C9081343C9000B4321200D
:109870002373FCF773FE854201D2122070BD2220B3
:10988000257AFCF76BFE8542F7D823781820042B45
:10989000F4D86378012BF1D80020EFE7030010B56E
:1098A0000220002909D0002B07D00322481C0A708F
:1098B00019000D3201F0A0FE002010BD03000222AD
:1098C000080010B5002B06D0002904D00E32591C18
:1098D00001F092FE0022100010BD030010B502201E
:1098E000002909D0002B07D00422481C0A70190057
:1098F0000C3201F081FE002010BD10B5FFF7DEFF35
:1099000010BD03000220002906D0002B04D0052240
:1099100000200A701B784B70704703000220002B58
:1099200008D0002906D05B7800200B70013B082B83
:1099300000D918307047030010B50220002909D063
:10994000002B07D00622481C0A7019000A3201F0C9
:1099500053FE002010BD10B5FFF7B0FF10BD020090
:109960000B00022010B500290ED0002A0CD00721D0
:109970001970118859701188090A997011180822F4
:10998000D81C01F039FE002010BD03000A0002209F
:1099900010B5002B0CD000290AD09978587809020C
:1099A00001431180901CD91C082201F025FE0020E3
:1099B00010BD030010B50220002909D0002B07D0EC
:1099C0000822481C0A701900921801F015FE0020A8
:1099D00010BD02000B00022010B500290BD0002A98
:1099E00009D009211970117818185970511C0622D4
:1099F00001F002FE002010BD10B5FFF75FFF10BDA3
:109A000002000B00022010B5002A09D0002907D05F
:109A10005178197011180622581C01F0EDFD002034
:109A200010BD030010B50220002909D0002B07D07B
:109A30000A22481C0A701900063201F0DDFD0020E0
:109A400010BD10B5FFF73AFF10BD02000B00022059
:109A500010B5002A06D0002904D018005178FFF76D
:109A600053FB002010BDF0B585B017001E006A46FC
:109A700006230500080091819380FEF7C0FC1324A3
:109A8000011E02900CD03800B047041E05D12800FA
:109A900001A9FEF76FFA041E02D0029801F074FECD
:109AA0002800FFF701FA200005B0F0BDF0B5040072
:109AB0008BB0019115000021102202A801F0CCFD0D
:109AC000334EA700B85900283CD0C388A34239D1EF
:109AD0000378002B36D14278062A18D10200010003
:109AE000553235310C3006ABFFF7A9FA002829D1E1
:109AF0002000FFF72FFE020006A902A801F07CFD5E
:109B0000200002A901F080FD01200BB0F0BD816EA4
:109B1000002917D00B8A112A28D19D420ED1019815
:109B20001231093A01F0E0FF012807D1BB592000AA
:109B30009D6EFFF70FFE29000200DEE732212000B4
:109B4000FFF7D8FC2000FEF701FF061E1BD0416A7C
:109B5000002918D00B8AAB4215D108220198123186
:109B600001F0C2FF01280ED1716A0AE09D42E9D1DD
:109B700008220198123101F0B7FF0128E2D1BB5948
:109B8000996E8A7EB9E7200001F07EFEBCE7C046F0
:109B9000D466FF1FF0B56B4D87007E5985B03378D2
:109BA00002900393002B00D087E0B368346A0193DE
:109BB0007078062817D101221B7D134202D0217B29
:109BC000114218D10222134202D0217B114251D1FD
:109BD0000422134203D0237B134200D08BE0019B6D
:109BE0005A7DEB5991E007380428F8D801F0BCFF02
:109BF000032E42678300B36E002B03D11C2001F0BB
:109C00004BFDB066EB599C6E002C1CD0102200213D
:109C1000200001F021FD0298FFF79CFD01002000CB
:109C2000FFF72DFA01F0D0FE20822000082112302B
:109C3000FFF725FA0298FFF78DFDA076EB5921007A
:109C4000D888FFF70FFC0822EB591CE0B36E002BFD
:109C500005D01A00198AF0881232FFF70DFC022293
:109C6000019B197DEB5911423DD0207B10423AD027
:109C7000073208E0F488FCF7DBFD01002000FFF765
:109C800011FC0A22EB595A70029B9C002A59537806
:109C9000073B042B11D8D088FEF758FE00284ED081
:109CA000C3895A08D2182849029B0298CB542B59D1
:109CB00041180433254801F0BFFE05B0F0BDFCF7A4
:109CC0009FFD03000120834201D100200393EB5943
:109CD000DE88FCF79BFD039902003000FFF7ECFBE8
:109CE000019AEB59117D042211420CD0217B1142C3
:109CF00009D00B22C7E7F688FCF73CFD01003000D5
:109D0000FFF7EEFB6BE7019A527D01210A4204D076
:109D1000607B084201D00C22B5E702210A4204D040
:109D2000607B084201D00E22ADE704210A4204D034
:109D3000627B0A4201D01022A5E71222A3E7FA2291
:109D40005200B0E7D466FF1FD866FF1F0BA10011B9
:109D500010B5064B1A780423100018401A4200D0A0
:109D60000348FFF727FA002010BDC0466165FF1FBA
:109D7000F843FF1F70B50400FFF7D4FA051E43D166
:109D80002000FFF77FFA234EA400A0598268937C3D
:109D9000DB0708D50321036A1B790B40012B02D195
:109DA000017F0B430377431DD97F8B1E022B0DD8F8
:109DB000022900D00121C088FCF790FF042133590B
:109DC0001A7F59700A431A77280070BD01290CD1F7
:109DD00002231022437000210C3001F03DFC305969
:109DE00010213530FFF74BF9EEE70529ECD10223BE
:109DF000D118437010220C3001F0FEFB04233259BD
:109E0000117F0B431377EAE708251828DCD1053DBD
:109E1000DAE7C046D466FF1FF0B58BB005914388E2
:109E20007E4F9E00F45915000493002C15D1012992
:109E300002D000200BB0F0BD101D57781678FFF748
:109E400057F9EB68320002932B7A04990193009042
:109E50003B002000FCF70CFFEBE7E388049A9342F9
:109E600001D00820E6E72378012B00D1D4E0059B40
:109E7000581E092800D9CFE001F076FE05CE0A2948
:109E8000CC506C859AB229000498FFF773FFD1E794
:109E9000200029001022453001F0AEFBB9594B7863
:109EA000042B02D1013B4B70C3E70B000A002533A2
:109EB00035320C310498FFF795F90498FFF702FA50
:109EC0000522431E9841BB59C0005A70B2E72000DA
:109ED00029001022553001F08FFB049B4F4C9D0050
:109EE000295904980A0006AB55320C31FFF77AF96C
:109EF00029591022453106A801F0F6FD012808D1A4
:109F00000498FFF7F7F90590002804D106222B5991
:109F10005A7005988EE708230593FAE763780C2BAF
:109F20007AD1E36E002B03D11C2001F0B5FBE06673
:109F3000BB59D86E00286FD01022290001F05CFBBD
:109F4000BB590498DC6EFFF705FC0D22A076BB59C7
:109F50005A706EE7E06E00285ED063780D2B5BD1FF
:109F60002B8808220382A91C123001F045FBBB5943
:109F70009A68517D0222114226D0186A407B104215
:109F800022D00C32E4E763780E2B45D1236F002BEF
:109F900003D1162001F080FB2067BB59186F002801
:109FA00003D01022290001F027FB0F22BB59CFE775
:109FB00063780F2B30D1206F0622691C103001F01E
:109FC0001BFBBB599A68517D0422114203D0196AC8
:109FD000497B1142D5D100210498FFF78BFA28E77D
:109FE000636F002B0DD0BB59586F0028F3D010229F
:109FF000290001F001FB0122BB5952425B6F1A613B
:10A00000E9E7142001F048FBBB5960675B6F002B48
:10A01000E9D126E72978DFE707200BE7D466FF1FA1
:10A0200010B5064C207001F067FC06212078FDF782
:10A0300091FF0348FEF778FC10BDC046E766FF1F9E
:10A04000C191001100200BB270B50D00834216DAE9
:10A05000264B187801F0D0FC041E0DD00378922B0B
:10A060000ED0A02B37D0224B1878FF283AD02100F1
:10A0700001F0C2FD002835D180200002684070BD8B
:10A0800043780E2B0BD03E2BEDD18378052B12D0CD
:10A09000082BE8D181798088FFF7D8FA08E0154BC2
:10A0A00082889A42DFD183681878591CFEF7C0FE77
:10A0B000002817D1D7E7104B1B785B0712D50F4B41
:10A0C0001B68002B0ED09B68002B0BD0C289811D12
:10A0D00080889847ECE7FFF741FAA068002801D094
:10A0E00001F052FB200001F0A7FAC5E7E766FF1F69
:10A0F000F143FF1F182000006165FF1FD066FF1F9E
:10A1000010B50078FFF712FA10BD10B50078FFF710
:10A11000FDFA10BD0C234343084A10B59B185A683A
:10A12000002A03D0012901D1904710BD9B68002B64
:10A13000FBD00029F9D19847F7E7C0460467FF1F15
:10A1400001238340094A10B5946B1C439463506B00
:10A1500098435063D46B20009843012901D120001B
:10A160001843D063116B0B43136310BD0080004094
:10A17000F0B500240127154B85B0DA6B144E03921D
:10A180001A6C0192DA64019BE3403B4217D0039DB5
:10A19000E5403D400295E5B202992800FFF7BAFF7D
:10A1A000316A736A002908D03900002B01D0029966
:10A1B00079402800FFF7C4FF01E0002BF9D10134FA
:10A1C0000C36172CDFD105B0F0BDC0460080004032
:10A1D000E866FF1F064B01215A68C2400A4204D0BC
:10A1E0001B68C3401800084070471B6DF9E7C04664
:10A1F000008000400122064B8240002903D0D9682C
:10A200000A43DA607047D9689143D960FAE7C046DB
:10A210000038004030B5032444430F4BE25C1B1967
:10A220009C785D7801232D1B0135AB40013BA34099
:10A23000A140DB430C00122807D8084992005218AD
:10A24000116819402143116030BD054A11680B4067
:10A2500023431360F8E7C0469BBE001108F000409E
:10A2600014F00040C21F70B5D4B20623092C0BD8DD
:10A270000125084C9540002908D00021FFF7CAFFAE
:10A2800023682B4323600023180070BD2368AB4371
:10A29000F8E7C04600380040214BF0B51B185B784A
:10A2A000022B21D1032444431E4A1F4EA35C1219E2
:10A2B0009478012215008540B76B013CE4B23D4320
:10A2C000A240B563194C122815D89B0000290CD167
:10A2D00017495B1899680A439A600123205C154A64
:10A2E000834011680B431360F0BD11495B189968F6
:10A2F00091439960F1E70E4B00290DD159690A434A
:10A300005A61225C1328E8D00123203A93400A497D
:10A31000086803430B60E7E7596991435961F0E727
:10A32000E866FF1F9BBE001100800040E0BE0011E8
:10A3300000F00040A0F00040A4F00040F8B5002478
:10A340001B4E1C4D1C4B1B5D012B1FD1194A9269E2
:10A35000E2401A420BD00122B25693402200143A36
:10A36000D2B2022A09D815494A6913434B61013414
:10A3700002360C35172CE5D1F8BD0022B2560F4934
:10A380009200521891680B439360F0E7022BEED1D4
:10A39000E7B23800FFF71EFF01235840C1B2380072
:10A3A000FFF77AFF3800FFF715FF6877DFE7C04651
:10A3B0006DBE0011E866FF1FE966FF1F00F0004058
:10A3C000012202388240054B002903D059690A4313
:10A3D0005A617047596991435961FAE70038004062
:10A3E000F8B50E0001210F008740114A0400D36820
:10A3F000FD43BB43D360831E8B4201D8FFF7E0FFD0
:10A4000000212000FFF72EFF0A4A0B4B5168012E56
:10A4100005D139431B1951605E700020F8BD2940F9
:10A42000516002221C1962709A6915409D61F4E71F
:10A430000038004000800040E866FF1F012210B590
:10A440008240074B002906D019680A431A6001218F
:10A45000FFF7C6FF10BD196891431960F7E7C046C2
:10A46000008000400C2370B5002543430A4A2900B0
:10A470009B181D70094B04001B185D70FFF7B0FF9F
:10A480000123A340064928000A681A430A600549C7
:10A490000A689A430A6070BD0467FF1FE866FF1FE1
:10A4A000348000403080004070B504000E00FF286A
:10A4B00013D003250540FFF7D5FF084AA3089B00EA
:10A4C0009B183F22ED00AA40AE401968200091433E
:10A4D000314319600121FFF78DFE70BD183800402F
:10A4E000F8B50C244443134B0500E4186368002BB3
:10A4F00003D1A3681220002B1AD0022201270E4B91
:10A5000000215B195A7028002770FFF769FF636804
:10A510001E1E08D0A3683E00002B04D02800FFF7C1
:10A5200059FE4640F6B228003100FFF709FE002030
:10A53000F8BDC0460467FF1FE866FF1FF7B5C420DB
:10A54000FF222B4B80001958002491433F3A0A43C5
:10A550001A508022274F5202274E1A60274B1D5D4A
:10A56000002D21D0A31E012B03D80121E0B2FFF75B
:10A5700027FF012D18D11F4B9B69E3402B4213D0BD
:10A58000E3B218000193FFF725FE01000198FFF7E1
:10A5900055FFE3B2143B022B1DD801217156184A16
:10A5A0008D405369AB4353613B7F002B0DD0E5B227
:10A5B0002800FFF795FF2800FFF70CFE7B7F0100C6
:10A5C000834202D02800FFF7A5FD01340C37023684
:10A5D000172CC3D1F7BD012100237156F3568D40CE
:10A5E000074A9B009B189A68AA439A60DCE7C0461A
:10A5F00000E100E0E866FF1F6DBE0011E966FF1F85
:10A6000000F0004070B50E0015000400FFF72AFFAF
:10A610000C236343094A20009B189D605E60FFF78E
:10A620005FFFF021064B074A8900051E5A5002D0F1
:10A630002000FFF717FF280070BDC0460467FF1F0A
:10A640000000FF1F71A1001170B5134D07202C7879
:10A65000002C1FD1982221005200280001F05CFA42
:10A660000123C420FF222B700C4B80001C635C6311
:10A670000B4B1C605C600B4B195891433F3A0A43EB
:10A680001A50802252021A600D20074A074901F031
:10A69000D3F8200070BDC046E866FF1F0080004070
:10A6A000A0F0004000E100E03DA500113DA3001135
:10A6B000030010B50620072B09D8054A137001F0D6
:10A6C00093FAD7210020034B034A89005A5010BD4A
:10A6D0002044FF1F0000FF1F911BFF1F70B51D00CE
:10A6E00002240C2910D8094ACA40D2070CD5FBF71E
:10A6F00041FF041E08D1059A04992800FBF756FF74
:10A70000FCF7C4FDFFF724FB200070BD1210000011
:10A7100030B50D7802232C009C43184201D02B4306
:10A720001C0008252300AB43284201D02B00234303
:10A7300020241D00A543204201D01C4325002A23CC
:10A740000D70184204D011781E3B0B43137030BDBE
:10A750000028FCD10C2113788B43F7E7F8B51D00D6
:10A7600006AB1B88140007AA0E000B201778002BDD
:10A7700027D10A78022A49D14A6850781178000214
:10A78000244A08438018042840D801F0EDF9031248
:10A790001D1B2300F06801F0EFF8021CC0B2B842A4
:10A7A00000D93A1CD2B22000F1682A8000F024FFC0
:10A7B00006E00222F3681B882A8023701B0A63705C
:10A7C0000020F8BD0622EEE701232B80F3681B78FA
:10A7D0002370F5E7F368002B16D008222A801A8828
:10A7E00022701A88120A62705A88A2705A88120A55
:10A7F000E2709A8822719A88120A6271DA88A271CC
:10A80000DB881B0AE371DBE72B80D9E701202B8073
:10A81000D7E7C04600D6FFFFF7B516000A781D003F
:10A8200008AB1F880C000123022A18D14A6850780F
:10A83000117800022B4A0843801803280FD801F032
:10A8400093F902254439E06801F096F8C0B2072375
:10A85000B84204D37B190193152B02DD0D23180098
:10A86000FEBDE0682A003100C01900F0C5FE6B464D
:10A8700000209B88E268D0541B4B1B68834203D0A6
:10A880001B68834200D098470023E8E70B23002F82
:10A89000E5D1022DE2D1737832781B021343E268CE
:10A8A0001380114B1B68002BEED01B68002BEBD0E4
:10A8B0000120E8E70B23002FD1D1062DCED12A00AD
:10A8C0003100E06800F098FEDEE70B23002FC6D1D0
:10A8D000012DC3D132787533012AC0D8E3681A70CC
:10A8E000D2E7C04600D6FFFFF468FF1F70B50C002A
:10A8F0001500072837D801F037F9041436361B360F
:10A90000242E182015290BD8184E162200213000AD
:10A9100000F0A2FE22002900300000F06DFE0020B1
:10A9200070BD18200229FBD11288114B1A80F6E75E
:10A9300018200829F4D10A000E48290001F094F8E3
:10A94000EDE718200129EBD10B4B10780B49DA69A0
:10A95000FFF7DEFEE3E718200129E1D1064B10786E
:10A960000749DA6BF4E70220DAE7C046DC68FF1F2C
:10A970009E44FF1F9444FF1F2444FF1F4C44FF1FAD
:10A980006C44FF1F030010B50020DB0704D507212E
:10A99000024A034800F08CF810BDC046F8BE001112
:10A9A0002444FF1F054A03001068002803D0828852
:10A9B0009A4201D1806870470068F6E7EC6AFF1F91
:10A9C0000A88030008009A4204D08A8804309A4218
:10A9D00000D0002070470000F8B5F22200230D4F90
:10A9E0000D4E7968050042433370994200D07B6078
:10A9F0000A4C0021200000F02FFE00231A007C608A
:10AA0000AB4202D100203370F8BD01332280DBB2AB
:10AA1000F234F5E7E46BFF1FE26BFF1FF06AFF1FE4
:10AA200073B56B4601900600684615001980FCF767
:10AA30005FFF041E11D1002D0FD07689002E11D09A
:10AA40000C2000F029FE00280ED0084A046013688C
:10AA500086808560002B02D11060200076BD1A0030
:10AA60001B68F7E70224F8E71324F6E7EC6AFF1FF8
:10AA7000012100220A4B10B549420A4C19809980E5
:10AA80009A719A70084B2070012019805A60FFF764
:10AA9000A3FF2078FCF78AFF0448FDF745FF10BDAF
:10AAA000FC68FF1FEC6BFF1FE46BFF1F5DAB001129
:10AAB000022310B5002802D0FFF7B2FF03001800F0
:10AAC00010BD0000030010B50020DB0704D50421F1
:10AAD000024A0348FFF7A4FF10BDC0460CBF001197
:10AAE000A444FF1FF0B50E2687B003930CAB1F885C
:10AAF00002ABF6180500080031000292FDF77AF863
:10AB000004000120002C0FD03088FFF74BFF03001A
:10AB10000E20002B08D05E68002E05D021002800F2
:10AB2000039B029A0097B04707B0F0BD0A4B10B5DF
:10AB3000984207D10122002352420A808B708A80FA
:10AB40008B7110BDFFF73CFF0028FAD001235B4258
:10AB5000038000238370F4E7FFFF0000F8B50500D1
:10AB600001290AD1134E00243388F227AB4219D0B1
:10AB700028001149FFF7DAFF06E0022904D1013964
:10AB8000FDF750FF0028EDD0F8BD3B00634372682D
:10AB9000D018D35A002B09D03A00002100F05CFDF8
:10ABA0000134E4B2054B1B78A342EED801235B428B
:10ABB0003380DDE7E46BFF1FFC68FF1FE26BFF1FC4
:10ABC00010B5FFF7FDFE03000020834200D0987807
:10ABD00010BD0000F0B589B01C000EAB80CB039017
:10ABE0001E8810AB1B78049202930B7A0D00DB06D3
:10ABF00016D42B780593022B24D00498FFF7D2FEAD
:10AC0000002812D003689C46002B0ED0029B220025
:10AC1000019329003B00644603980096A04705E095
:10AC20000498FFF7BFFE002802D10E2009B0F0BD46
:10AC30008368002BF9D00A2229000398984700283E
:10AC4000D7D0F3E76B6858781A786B4B0002104343
:10AC50009842D2D8043B984210D2684B984242D0D6
:10AC600015D8674BC0180128C7D80B20002EDDD19E
:10AC7000EB681A7859683A80200028E0614BC018C8
:10AC8000032800D979E000F06FFF846A789E5E4B5C
:10AC90009842B2D10B20002EC8D101233B80EB6833
:10ACA00031001B7823706889013080B2FCF7A2FF65
:10ACB0003A88031E0ED0017802328A183A804289FF
:10ACC00062704289120AA27059680278E01C00F092
:10ACD00093FC06E004323A8031000422601C00F04C
:10ACE000BBFC0020A2E70B20002E9FD1EB6807A938
:10ACF0001E8804233B80330A300026706370FCF703
:10AD000079FF051E28D004AB9A890E2304A95B188D
:10AD10003E49C668FCF7E2FF00280BD12B783C487F
:10AD20006A680599FBF798FB002803D1012304AA60
:10AD30005B42D3813278022A06D17168201D00F06F
:10AD40005BFC3B8802333B800E2304AA9B181B88C4
:10AD5000A3701B0AE370C4E704ABDE81F4E70B20A9
:10AD6000002E00D062E7E9680398FFF729FF02236D
:10AD70003B802070000A6070B3E70B20002E00D0EB
:10AD800054E70222EB681B883A8023701B0A637029
:10AD9000A7E7E86800F0F0FDC2B203000720B24266
:10ADA00000D243E70DD00299DBB27118994202DB61
:10ADB000921BD3B20293029BE9681A003B80891967
:10ADC0005AE70023F6E70B20002E00D02EE70722DB
:10ADD000EB683A801A7822705A7862705A88A270AA
:10ADE0005A88120AE2701A792271DA886271DB8855
:10ADF0001B0AA37175E7C046042900000228000061
:10AE000000D8FFFFFFD6FFFF03280000FFFF000070
:10AE10003CBE0011F0B58DB06B4600200891202299
:10AE20009B5E83423DDAA64B187800F0E5FD071ED5
:10AE300032D00378B02B2CD10079023816281FD8D5
:10AE400000F04AFD17001E001E001E0031001E000B
:10AE500096001E001D011E0052011E0073011E00FF
:10AE6000CD011E0050021E001E001E008E021E009C
:10AE7000E302944B94491B8878880B80FBF72CF8ED
:10AE80003800FCF7ADFF914B1B68002B01D0380058
:10AE90009847380000F0D0FB8020089B0002434018
:10AEA00018000DB0F0BDEE220021874800F0D4FB61
:10AEB0000BAA3B7B7989388900923A000D32FCF766
:10AEC000B1FD0400804B1B78002C3FD146E0804B45
:10AED000788805937F4B4100CB5A0BAE073BDBB222
:10AEE00032880293002301937B4B21000693009349
:10AEF000059BFFF76FFE744D002810D1069B3A8A20
:10AF00001B889A420BD138000599123000F0ECFDF5
:10AF1000002804D02B7862899B00EB185A801623F6
:10AF200006A81B18328820007989FCF7D7FE2B78F9
:10AF300004009A00AA1851880029C3D00133DBB25B
:10AF40002B70002807D006A9C98A9180634A12880D
:10AF50009A42BCD802E0012149429180002B04D0E2
:10AF600059497888FAF7ECFF8AE73E890A2479E0A4
:10AF700000253E89574B06937B88069A5B009B5AB7
:10AF8000033B9D4202DB002DF0D05BE0162206A8B9
:10AF900012183B7B798900923A0030000D32FCF7A1
:10AFA00041FD0590002858D04689017A7888FCF741
:10AFB00003FD041E44D1464B78880793069B41004D
:10AFC000C95A454B0439C9B206AAD28A06930291DE
:10AFD000019400930599079BFFF7FCFD041E2FD1F8
:10AFE000069B39491A88931C002D26D14B807988FD
:10AFF000384B4900CB5A5119033B8B4220DD059B4E
:10B0000031485B8941190B71A91C0135C9B2EDB2F8
:10B01000059145191B0A2B71059B2D4904331818FE
:10B0200000F0EAFA2C4B059A1B88D318DDB22C4BA2
:10B030009E4205D00136B6B29CE749889942D6D0E7
:10B04000002D0CD0204C2800618800F0B5FA20704B
:10B0500021007888FAF784FF12E7059CF0E7002CBE
:10B0600000D183E77B78142B00D109E716493B799F
:10B070004E800B700C717888FAF724FF00E71624D5
:10B0800006ABE41821003889FCF7B4FD011E00D19D
:10B09000B7E1788822880F4C45002C5B0A4D013CB3
:10B0A000E4B2029400240F4B01940095FFF792FD47
:10B0B000041E00D014E129007888FAF761FFDFE66A
:10B0C000EC6BFF1F9043FF1F0469FF1FF868FF1F11
:10B0D000F869FF1F3465FF1FE86AFF1F8E43FF1FDB
:10B0E000FFFF00000669FF1F162406ABE4182100CD
:10B0F0003889FCF77FFD011E00D182E17888228823
:10B10000AE4C45002C5BAE4D013CE4B202947C8910
:10B11000AC4B01940095FFF75DFD041E00D0DFE00D
:10B1200029007888FAF736FFAAE60025A44B1D808F
:10B130003B00F6331B78A24A78880792AB4208D9C5
:10B140009E4B12880693069943005B5A013B9A4234
:10B1500003DB0799FAF728FF92E616246B00FB1829
:10B16000059306ABE418059B21001889FCF742FD06
:10B17000011E03D1059B01241E8973E77888924B39
:10B180002288069C099343001B5B904E013BDBB277
:10B190000293002300960193099BFFF71BFD041EF9
:10B1A00002D0059B1E895DE77B88069A5B009B5A4F
:10B1B000079A108832881218934202DC1B1A013B4E
:10B1C00033807F4C023032880999001900F014FA5C
:10B1D0002388328801359B182380EDB2A8E70BAA9B
:10B1E0003B7B7989388900923A000D32FCF71AFCD2
:10B1F00000250590059B002B04D10A24002D00D1C9
:10B200006EE060E0059B7888197AFCF7D5FB0100B9
:10B21000041E63D1694C6C4B788806940993069B95
:10B220004400E45A694B063CE4B20BAE3288079303
:10B230000294019100930599099BFFF7CBFC041E32
:10B240004CD1079B5E491B881A1D002D30D14A80C6
:10B25000059B5B4C5A8963191A716B1C9BB2E318EE
:10B26000120A1A71162306A832881B1879890598C4
:10B27000FCF734FDFF21AA1C2E1D03350B000590A1
:10B2800092B2B6B2ADB2002803D006ABDB8AD9B217
:10B290001B0AA218651911712B714C4D301D2A889B
:10B2A0004949201800F0A8F92B88F618B5B2A1E793
:10B2B0004988914207D17A8806995200525AEB1870
:10B2C000053A9A42C4DC3E4C2800618800F0BCFA82
:10B2D000207021007888FAF771FED1E5002DF2D1B7
:10B2E0003E89BFE6162606ABF61831003889FCF712
:10B2F00081FC3D000400FA3500282DD0037A9B061E
:10B300000CD400227B893989788800923A000C326B
:10B31000FFF7E8FB041E10D03E8915E03088FFF7E8
:10B3200041FB00281AD08368002B17D0210012227D
:10B3300078889847041EE4D0EEE72B78002B02D1E2
:10B340007888FAF74BFE00262B78002B00D097E583
:10B35000002C00D194E585E60124DDE70E24DBE72F
:10B36000162506ABED1829003889FCF743FC041EAE
:10B3700047D0037A9B0611D4154A7B8811889942DD
:10B3800003D01448814207D11380134BF2261D7855
:10B390000023D9B2A94221D30924A1E72888FFF7C5
:10B3A00001FB00282FD08368002B2CD02100122213
:10B3B00078889847041EDFD092E7C0463465FF1FA7
:10B3C0000469FF1F0669FF1FF869FF1FE86AFF1F76
:10B3D000E46BFF1FFFFF0000E26BFF1F31005943CA
:10B3E000546801336018615A0029D2D13C000834F6
:10B3F0002100F22200F000F921007888FAF7F6FD2A
:10B400003EE501246CE70E246AE71D4B1A887B8811
:10B410009A4231D07888FAF7F3FD31E5F2230598A6
:10B4200051684343CD18C95A00291FD03B7A012BDC
:10B430000BD16C88AB887888AA1D0094FFF752FB6B
:10B44000041E02D000233B722E88F2220021280025
:10B4500000F002F900232B80059B0133DBB205933A
:10B46000084B05991B78064A8B42D7D801235B42CB
:10B470001380002CCED0F5E5002634000596EFE7CA
:10B48000E46BFF1FE26BFF1F70B504000E00150098
:10B49000FFF796FA031E08D131000548FFF790FA2E
:10B4A00003001120002B02D01C8000209D7070BD75
:10B4B000FFFF0000F8B50B4F06003B780D001400AD
:10B4C000FF2B0ED00A2000F05FFB011E09D0B12334
:10B4D0000380002346800371C5800481387800F022
:10B4E0008BFBF8BDE544FF1FF7B50F0008A9060068
:10B4F000088809A90B240988002821D10234022BCD
:10B500001ED1557813782D021D432B008B430193D8
:10B510007334002B14D1FB68300019000093FFF73F
:10B520004FFB019C85420BD02A0030000099FFF7A9
:10B53000ABFF041E04D12A0030007989FFF7BAFF5F
:10B540002000FEBDF0B50E7885B003900AA80588EE
:10B550000120022E0DD14C682778647824023C43E8
:10B56000054FBC4205D10398DBB201960095FFF769
:10B57000BBFF05B0F0BDC04602290000034B10B56B
:10B580001B68002B00D09847FEE7C046F06BFF1FFA
:10B5900007B501A8FFF7F2FF044A05480021121A77
:10B5A00000F0BAFAF8F726F9FEE7C046F46BFF1F81
:10B5B000E844FF1F0000000001B40248844601BCBB
:10B5C000604700BF350E000001B40248844601BC4C
:10B5D000604700BFDD66010001B40248844601BC3B
:10B5E000604700BFE548000001B40248844601BC42
:10B5F000604700BF291C000001B40248844601BC1A
:10B60000604700BFE94C010001B40248844601BC18
:10B61000604700BF311B000001B40248844601BCF2
:10B62000604700BF4550000001B40248844601BC99
:10B63000604700BF014C010001B40248844601BCD0
:10B64000604700BF434D010001B40248844601BC7D
:10B65000604700BF4551010001B40248844601BC67
:10B66000604700BF154D010001B40248844601BC8B
:10B67000604700BF4D1F000001B40248844601BC72
:10B68000604700BF851F000001B40248844601BC2A
:10B69000604700BF0919FF1F01B40248844601BC7E
:10B6A000604700BF3D4B010001B40248844601BC25
:10B6B000604700BFB14E000001B40248844601BC9F
:10B6C000604700BF8B52010001B40248844601BCB0
:10B6D000604700BF1D4B010001B40248844601BC15
:10B6E000604700BFBD39FF1F01B40248844601BC5A
:10B6F000604700BF7936FF1F01B40248844601BC91
:10B70000604700BFE117000001B40248844601BC55
:10B71000604700BF156B010001B40248844601BCBC
:10B72000604700BF2526000001B40248844601BCE2
:10B73000604700BFB54C010001B40248844601BC1B
:10B74000604700BFF94C010001B40248844601BCC7
:10B75000604700BF6571010001B40248844601BC26
:10B76000604700BF017F000001B40248844601BC6D
:10B77000604700BFADAE000001B40248844601BC82
:10B78000604700BF3519FF1F01B40248844601BC61
:10B79000604700BFD949010001B40248844601BC9A
:10B7A000604700BFF138FF1F01B40248844601BC66
:10B7B000604700BF1147010001B40248844601BC44
:10B7C000604700BF5522000001B40248844601BC16
:10B7D000604700BFC9A9000001B40248844601BC0B
:10B7E000604700BF0D52010001B40248844601BC0D
:10B7F000604700BF8D12000001B40248844601BCBE
:10B80000604700BFD91B000001B40248844601BC58
:10B81000604700BF5952010001B40248844601BC90
:10B82000604700BF9130FF1F01B40248844601BC4D
:10B83000604700BF2146010001B40248844601BCB4
:10B84000604700BF1931FF1F01B40248844601BCA4
:10B85000604700BF090E000001B40248844601BCE5
:10B86000604700BF1134FF1F01B40248844601BC89
:10B87000604700BF5147010001B40248844601BC43
:10B88000604700BFC56D010001B40248844601BC99
:10B89000604700BF091B000001B40248844601BC98
:10B8A000604700BFC521000001B40248844601BCC6
:10B8B000604700BFFD37FF1F01B40248844601BC4A
:10B8C000604700BF056A000001B40248844601BC1D
:10B8D000604700BF0539FF1F01B40248844601BC20
:10B8E000604700BFF93BFF1F01B40248844601BC1A
:10B8F000604700BF75A9000001B40248844601BC3E
:10B90000604700BFC926000001B40248844601BC5C
:10B91000604700BF7918000001B40248844601BCAA
:10B92000604700BFEDA5000001B40248844601BC99
:10B93000604700BFC51D000001B40248844601BC39
:10B94000604700BFD13BFF1F01B40248844601BCE1
:10B95000604700BFE928000001B40248844601BCEA
:10B96000604700BF5536FF1F01B40248844601BC42
:10B97000604700BF293AFF1F01B40248844601BC5A
:10B98000604700BFDD52010001B40248844601BC9B
:10B99000604700BF055E000001B40248844601BC58
:10B9A000604700BF3D39FF1F01B40248844601BC17
:10B9B000604700BF3D18000001B40248844601BC46
:10B9C000604700BF3555000001B40248844601BC01
:10B9D000604700BF2951010001B40248844601BC00
:10B9E000604700BFED4A010001B40248844601BC33
:10B9F000604700BFC94A010001B40248844601BC47
:10BA0000604700BFF54E010001B40248844601BC06
:10BA1000604700BF4936FF1F01B40248844601BC9D
:10BA2000604700BF8552010001B40248844601BC52
:10BA3000604700BFA54F010001B40248844601BC25
:10BA4000604700BFA946010001B40248844601BC1A
:10BA5000604700BF5125000001B40248844601BC84
:10BA6000604700BF9DA9000001B40248844601BCA4
:10BA7000604700BF810E000001B40248844601BC4B
:10BA8000604700BF456B010001B40248844601BC19
:10BA9000604700BF312EFF1F01B40248844601BC3D
:10BAA000604700BF4937FF1F01B40248844601BC0C
:10BAB000604700BF7930FF1F01B40248844601BCD3
:10BAC000604700BF7D39FF1F01B40248844601BCB6
:10BAD000604700BF350E000001B40248844601BC37
:10BAE000604700BFE132FF1F01B40248844601BC39
:10BAF000604700BFCD4C010001B40248844601BC40
:10BB0000604700BF0124000001B40248844601BC24
:10BB1000604700BFA53AFF1F01B40248844601BC3C
:10BB2000604700BFB70E000001B40248844601BC64
:10BB3000604700BF6DBC000001B40248844601BCF0
:10BB4000604700BF2124000001B40248844601BCC4
:10BB5000604700BFD13AFF1F01B40248844601BCD0
:10BB6000604700BF5D17000001B40248844601BC75
:10BB7000604700BFE53BFF1F01B40248844601BC9B
:10BB8000604700BF691F000001B40248844601BC41
:10BB9000604700BF1D4D010001B40248844601BC4E
:10BBA000604700BF5549010001B40248844601BC0A
:10BBB000604700BFB352010001B40248844601BC93
:10BBC000604700BFF30E000001B40248844601BC88
:10BBD000604700BF090E000001B40248844601BC62
:10BBE000604700BFB932FF1F01B40248844601BC60
:10BBF000604700BF911BFF1F01B40248844601BC8F
:10BC0000604700BF594F010001B40248844601BC9F
:08BC1000604700BF7D2EFF1FFD
:10BC180000030102020303030403050006020700F0
:10BC2800080209030A030B030C000D000E030F039F
:10BC3800100311031303140315021602993B001194
:10BC4800CD3B001100000000020000005ABC0011AA
:10BC5800192A0F180A000000F1590000FD240000FD
:10BC6800414601003180001145A00011997400116E
:10BC7800357E00111153001115AE00115D4F0011F2
:10BC8800A93D0011D93E0011000000001616000061
:10BC980002000000A4BC0011F4FFF3FFD2FC000076
:10BCA800194000110000000000000000547579617F
:10BCB8000042312E340030303137006769746875BE
:10BCC800622E636F6D2F707676780054484231008B
:10BCD80002000000ECBC0011292A282A272A262A5B
:10BCE800252A242A0A180000E20400007102000034
:10BCF80078EC0000744000001027000060F000009D
:10BD080006640000204E000000000000050000004E
:10BD18001F501D00023CB400000117001400000071
:10BD2800A1020000303132333435363738394142D8
:10BD3800434445460000000015570011695700119B
:10BD4800000000000200000058BD00116F2A6E2A92
:10BD58001A18EAD8BC80F0FC60000000000000005F
:10BD680000005F066B2F363D7D077F3F777C596E5D
:10BD78007971000001A00000000000006410B71DE8
:10BD8800C8206E3BAC30D9269041DC76F4516B6B01
:10BD98005861B24D3C7105502083B8ED44930FF0C3
:10BDA800E8A3D6D68CB361CBB0C2649BD4D2D38679
:10BDB80078E20AA01CF2BDBDFB349B5F80000080C6
:10BDC80000100000000000009B60001125770011A2
:10BDD800BF6000112D7B001143610011037B00112E
:10BDE800B9610011D97A00110B620011A17C001110
:10BDF80073620011A17C0011A56200115B7C001127
:10BE0800B9610011917A001131620011397C001179
:10BE1800000000000000000017630011397C0011C9
:10BE2800796300113D770011052A042A012A002AA6
:10BE38000229032801280028011800180000000022
:10BE4800000000000000000000000087010102015E
:10BE580002010102010203030401030101010101BE
:10BE68000303020103000D000E001000110013006F
:10BE78001401070108010A010B011C011D0204023B
:10BE880005020702080219021A021C021D03010317
:10BE9800020317000201000504000807000B0A004E
:10BEA8001716001D1C010201010504010E0D0111E8
:10BEB80010011413011716011A19020201020B0AC4
:10BEC800020E0D02111002141302171603050403C3
:10BED8000807030B0A030E0D0001020307090A0BEA
:10BEE8000E0F101112141718191A1B1F20212200E7
:10BEF8005DA7001119A80011000000000200000051
:10BF080042BE00110000000045B50011000000000D
:08BF18000200000040BE001110
:020000041FFFDC
:1000000000000000113D001160BC00115CBC00113B
:100010001862FF1F00000000000000000000000048
:1000200000000000000000000000000000000000D0
:1000300000000000000000000000000000000000C0
:1000400000000000000000000000000000000000B0
:1000500000000000000000000000000000000000A0
:100060000000000000000000000000000000000090
:100070000000000000000000000000000000000080
:100080000000000000000000000000000000000070
:100090000000000000000000000000000000000060
:1000A0000000000000000000000000000000000050
:1000B0000000000000000000000000000000000040
:1000C0000000000000000000000000000000000030
:1000D0000000000000000000000000000000000020
:1000E0000000000000000000000000000000000010
:1000F0000000000000000000000000000000000000
:1001000000000000000000000000000000000000EF
:1001100000000000000000000000000000000000DF
:1001200000000000000000000000000000000000CF
:1001300000000000000000000000000000000000BF
:1001400000000000000000000000000000000000AF
:10015000000000000000000000000000000000009F
:10016000000000000000000000000000000000008F
:10017000000000000000000000000000000000007F
:10018000000000000000000000000000000000006F
:100190000533FF1F6531FF1FC1660100000000002D
:1001A000000000000000000000000000000000004F
:1001B000000000000000000000000000000000003F
:1001C000000000000000000000000000000000002F
:1001D000000000000000000000000000000000001F
:1001E000000000000000000000000000000000000F
:1001F00000000000000000000000000000000000FF
:1002000000000000000000000000000000000000EE
:1002100000000000000000000000000000000000DE
:1002200000000000000000000000000000000000CE
:1002300000000000000000000000000000000000BE
:1002400000000000000000000000000000000000AE
:10025000000000000000000000000000000000009E
:10026000000000000000000000000000000000008E
:10027000000000000000000000000000000000007E
:10028000000000000000000000000000000000006E
:10029000000000000000000000000000000000005E
:1002A000000000000000000000000000000000004E
:1002B000000000000000000000000000000000003E
:1002C000000000000000000000000000000000002E
:1002D000000000000000000000000000000000001E
:1002E000000000000000000000000000000000000E
:1002F00000000000000000000000000000000000FE
:1003000000000000000000000000000000000000ED
:1003100000000000000000000000000000000000DD
:1003200000000000000000000000000000000000CD
:1003300000000000000000000000000000000000BD
:1003400000000000000000000000000000000000AD
:10035000000000000000000000000000000000009D
:10036000000000000000000000000000000000008D
:1003700091B5001100000000000000000000000026
:10038000000000000000000000000000000000006D
:10039000000000000000000000000000000000005D
:1003A000000000000000000000000000111BFF1F03
:1003B000000000000000000000000000000000003D
:1003C000000000000000000000000000000000002D
:1003D000000000000000000000000000000000001D
:1003E000000000000000000000000000000000000D
:1003F00000000000000000000000000000000000FD
:081838000070FF1F4118FF1FA3
:10184000024981F3088802F003FC00000070FF1FCA
:1018500070B500241E491F4A1F484C6308CA1B0567
:101860001B0DE4188242F9D11C4B80228B630021AE
:1018700009201B4B920519621A4B1B4DDA671B4B53
:10188000DA688243DA609A68194802409A60112047
:10189000296002F093F8112002F070F86B6C154A81
:1018A000112013406B64EE23DB006343124A1B0CD0
:1018B00013840122114B9A7201F00AFC104B1B7821
:1018C000002B04D10F4B1021187802F029FA70BDBB
:1018D000000005400806054080060540FF010000A5
:1018E00000F0004004E100E0003800403CF000401F
:1018F000FFDFFFFFFFFEFFFFE861FF1F9C62FF1F8E
:10190000CA64FF1FC862FF1F10B502F079FB0728E9
:1019100004D0122808D0022808D010BD044A0420A0
:10192000136B01331363F8E70220F6E71420F4E7A2
:10193000DC65FF1FF8B507000C00260025005036B7
:1019400030785135002804D10300287058342370B2
:10195000F8BD2978CA00481E8141A3183800A25C4E
:101960005B68C9B2FFF7D0FF00280DD12B78DA00F1
:10197000A218013350602B703378044A013B337056
:10198000136A01331362D8E70123DFE7DC65FF1F29
:101990005C234343074910B5C9180B0058331B7823
:1019A000012B05D1FFF7C6FF034A936A0133936207
:1019B00010BDC0461066FF1FDC65FF1F10B502F0AA
:1019C00057FB064A0121130010CB4942D967044B4B
:1019D000136002F015FA200010BDC04600E100E0DF
:1019E0001000100010B5040002F042FB024B1C6016
:1019F00002F006FA10BDC04600E100E0431E5A4264
:101A00005341A022F0B5D2015B421340154D164A56
:101A100040019B182A18127E8BB00191002A1BD01E
:101A20001A000832D46F0022E6B206AFE4B2944244
:101A30000EDC2818C369002B08D0019902AA117185
:101A400006AA049202AA167303A898470BB0F0BD29
:101A50001978B9540132EAE71A7D1A7806AB0126E3
:101A60001A70E6E79C68FF1F00400040F0B5254B68
:101A700004004001C25C85B0002A2BD01A18117EE8
:101A8000002927D0917E002924D01179022921D163
:101A90001689D788D168F51BADB22A1C102D00D944
:101AA000102292B2BE4217D11818012303710023ED
:101AB000C269C38003819A4206D06846032103733A
:101AC0000171029301A890470820002C00D0192032
:101AD00001F0FEFA05B0F0BD013C65426C41A02565
:101AE0006442ED012C40084D1B186419074D063364
:101AF000013A92B2AA42EDD01888461C1E80085CBA
:101B00002070F5E79C68FF1F00400040FFFF0000C9
:101B10000F220E4B10B59868104002380A280BD8D7
:101B200002F060F80D0A0B0A0A110A0A0A0A0600F6
:101B300002210020FFF762FF10BD0121F9E700201C
:101B4000FFF794FFF8E7DB6FF6E7C0460040004080
:101B50000F220E4B10B59868104002380A280BD897
:101B600002F040F80E0A0B0A0A120A0A0A0A0600D4
:101B700002210120FFF742FF10BD01210800F9E713
:101B80000120FFF773FFF7E7DB6FF5E700900040F8
:101B900013B5334C2378072B3DD8324B1A78324B90
:101BA000002A39D18022196852020A431A6025207E
:101BB00001F0C4FE20232D4A11680B4380211360DD
:101BC0006B460422C90508680733104228D08021DB
:101BD0000422C905C86810422ED080212020C905E2
:101BE000CA688243CA6014221A701A78002A2FD158
:101BF0008021C905C86820320243CA6014221A70C5
:101C00001A78002A28D11A4B1A7D22785A601D2290
:101C10001A705932DA6013BD1A6816490A40C5E7CE
:101C2000086802430A6014221A701A78002ACED07B
:101C30001A78013AD2B2F7E7C8680243CA601422A0
:101C40001A7019784A1ED2B21A700029F9D1C4E765
:101C50001A78013AD2B2C7E71A78013AD2B2CEE77F
:101C60002044FF1FE844FF1F3CF000401844FF1FC2
:101C700000200040FFFFFEFF564B70B51B68012B94
:101C800003D1554A936D0133936502F059F8534BD4
:101C9000534A1860534B544C1A600123534A136043
:101CA000534A13602378002B06D00622514952482C
:101CB00002F06EF900232370504A514B10681B78D4
:101CC000C1B2002B0ED14F4CC0B223785BB2002BB7
:101CD0004FDB237824785BB264B21B0424021B1907
:101CE0001B1813600B1C50294ED95023464A4749F4
:101CF0001078DBB2FF2202284BD10868444C454DD6
:101D0000267890432A78964254D9227824782E78DF
:101D1000023B5D10A31B6B435201D31A10335B11BE
:101D20001843086002F03CF8031F012B45D83A4BDA
:101D30001B78002B06D0394B1B78002B02D00020DB
:101D400002F01EF9A122364B92009978354B4A4396
:101D50001B689B18832292009B181B78033B012B66
:101D600003D8AF20400002F0EBF801222E4BDA82BC
:101D700070BD237824785BB264B2FF33FF341B0458
:101D800024021B190138ABE7CAB2022AAED20223E1
:101D9000ACE70868254C264D267890432A78964271
:101DA00008D9227824782D78023B5B10641B6343AA
:101DB0005201B2E72378DBB2B2E70228D5D11D4B3E
:101DC0001B78013B022B03D91B4B1B78022BCCD178
:101DD0006C20C8E79809FF1FFC0FFF1F1465FF1F49
:101DE000FF3F0000141003401865FF1F0C10034054
:101DF00000100340D50BFF1F7211FF1FB4000340FA
:101E00008C09FF1F680AFF1F490AFF1F9400034047
:101E1000460AFF1F470AFF1FF908FF1F2209FF1F7D
:101E2000300DFF1F3409FF1FBC0BFF1F440AFF1FAB
:101E3000450AFF1F1C09FF1F2309FF1F10B501F0F2
:101E40005FFF0022014B1A8010BDC0461265FF1FC4
:101E500010B501F0B5FFA121054A89009478054A23
:101E600061431268044B5218528C1A8010BDC04650
:101E7000300DFF1F3409FF1F1265FF1F10B50D4BFA
:101E80000D4A9978A1239B004B431268D218531D29
:101E9000D97F0A4B1B88994209D2441C07D0C82815
:101EA00005D0D2695B1A5A43054B5343C01802F060
:101EB000F7F810BD300DFF1F3409FF1F1265FF1F1B
:101EC0007102000070B5244D2B68002B28D001F062
:101ED000D7FF2B68D8402B680400002B27D001F0D7
:101EE0009FFE2B68D8401D4B1D4A9978A1239B006B
:101EF0004B431268D118D25C91239B00002A20D05A
:101F0000CA580132CA50174B17491B6808688342E8
:101F100014D3D23B181A012A1AD0144B186070BD82
:101F200001F0AEFF124B196801F0BAFED3E701F0E1
:101F300077FE0F4B196801F0B3FED4E70D495B182B
:101F4000E8E7CA500C4B1B68DB68E418201AE4E78A
:101F5000F530FF30E1E7C0461C08FF1F300DFF1FC2
:101F60003409FF1F9C09FF1F1465FF1FA009FF1FF5
:101F70001808FF1F2DFF3F001C65FF1F70B50400F0
:101F80000D00282916D10300A433C2881B889B1A90
:101F90000B4A9BB293420DD906006A3605223100E6
:101FA000653001F085FE002804D13100200002F0E8
:101FB00087F870BD2900200001F0D2FEF9E7C04685
:101FC000FE7F0000F8B50500012001F0A9FF134CC9
:101FD000A36AA26A9342FBD1114E336001F020FF45
:101FE0001049030008601048426894460F4A176879
:101FF0000022BC4501D24268BA1A0D48026032681C
:10200000AD18A422E562606A520302436262094A83
:102010001278002A01D00F3B0B60F8BD00F00040A1
:10202000340AFF1FE408FF1F28100040180AFF1F92
:102030001C0AFF1F1C09FF1F70B580241025E40532
:10204000A3682B43A36001F003FFA368AB43A36025
:1020500070BD0000F7B5160080221C001023D205C9
:102060000191916805000B43936000225A4BD730D1
:102070001A6001F0B5FE9D232A002F009B00EB584B
:10208000CA3201210092FC37002B01D00021009AB6
:10209000386801F075FE2900009BCB311A784F4B50
:1020A000D3351A604B780A781B0213438A781204DE
:1020B0001A43CB781B061343494A1BBA13604B796A
:1020C0000A791B0213438A7912041A43CB7931002F
:1020D0001B061343434A1BBA13606B782A781B0212
:1020E0001343AA7812041A43EB781B0613433E4AA3
:1020F0001BBA1360019A330213433C4A13603C4BF2
:1021000022001B1B9C4603293DDCB3089A001300E8
:102110005142B21A032A46D1354AE018511A827840
:102120004078120400020243E05C043302430A6078
:102130000022FF2B4BDDF0222E4B12011A600F22E2
:102140002D4B1A602D4A1368002BFCD00023224A25
:1021500027491360091B321D0B191B68043A180A22
:1021600023706070180C1B0EA070E3700434002AFA
:10217000F2DC802210213B68D20501333B6093687A
:102180008B439360F7BD6346D578981893782D06F6
:102190001B042B43157804392B43557804322D0248
:1021A0002B430360AFE7022A0AD1114AE05C511ABF
:1021B000E2185278120202430A6004339BB2B7E776
:1021C000012AB5D10A4A521AE15C1160F5E70849C3
:1021D00059180A600433ACE7000004403C00044096
:1021E0003800044034000440300004400C00044037
:1021F00000010440040004401000044014000440A6
:10220000F7B5150080221C001023D20500919168BB
:1022100007000B4393600023654AD730136001F039
:10222000DFFD9D233E009B00F9583B00CA3632007B
:10223000FC33002900D07FE0586801F0A1FD39008F
:1022400032785C4BCB311A604B780A781B0213430F
:102250008A78AC4612041A43CB78281D1B06134318
:10226000554A1BBA13604B790A791B0213438A79CA
:1022700012041A43CB791B061343504A1BBA13604E
:102280004B7A0A7A1B0213438A7A12041A43CB7AD6
:1022900021001B0613434A4A1BBA1360009A2B0203
:1022A0001343484A13602200474B1B1B0093009BBB
:1022B000CE785B1801938B7836061B0433430E7877
:1022C000043833434E78043136023343019E336081
:1022D0000328ECDC0321A808431C9B002940800054
:1022E00003292BD13849E5185E18A9786D78E35C8D
:1022F00009042D02294319433160030008330021EA
:10230000FF2B2DDD314B324919600F21314B196004
:10231000012327490B60304B19680029FCD00621A6
:102320001B680B40042B20D080220020D20593682C
:102330000A318B439360FEBD01217DE7022908D15C
:1023400021495D18E1184978E35C090219432960C5
:10235000D3E70129D3D11C495918E35C0B60CCE7C2
:102360001948181801600433CAE7002310490B60AC
:102370006346002B0CDC3B00FC335A681021013211
:102380005A608022D205936801208B439360D2E784
:10239000009B9B181B68190A13705170190C1B0EB7
:1023A000D37004235B4291709C440432E0E7C04642
:1023B000000004403C000440380004403400044065
:1023C000300004400C0004400001044004000440BC
:1023D000080F0000100004401400044070B5061EF1
:1023E00019D002225A4B9B799343012B13D1594B9D
:1023F0001A78FF2A0FD15A78FF2A0CD19A78FF2A2F
:1024000009D1DA78FF2A06D11A79FF2A03D15B793C
:10241000FF2B00D199E0504B0C201A78012A08D0EC
:1024200000224E4D1A7029780B00093B042B01D86D
:10243000212070BD4B1F012BFAD9454CA37B042BE7
:1024400000D982E0A279032A00D97EE09A1ED2B296
:10245000012A02D860881F2877D9002E56D0012E75
:1024600073D1A0880128E3D0002907D1581E032882
:1024700003D801F0B7FB121715122E702978481EE9
:10248000032811D80025364B1D602823237501F041
:102490006FFDA84227D0A580CAE702212970EDE789
:1024A0000421FBE70321F9E707390129C0D82D49A9
:1024B0000968C96A8906BBD52B4908780028B7D1B5
:1024C000012A01D9002BB3D102230B708021274DA3
:1024D000263389012878237501F0F2FB80212878C2
:1024E000890101F01DFC0123A380214B1B78002BE7
:1024F0000AD0FA2280211F4B92001B8809025A43FE
:102500001A4B187801F074FC002092E701F0B0FD3E
:102510002B78A680073B012B03D917482E7001F0BA
:1025200017FD114B114C1A78002A06D08021002289
:10253000207889011A7001F0C3FB01F061FC802151
:102540002078090201F0BCFBDEE7122071E7C046EB
:10255000A60BFF1F6B09FF1F1A09FF1F1C09FF1F96
:102560004809FF1F1C65FF1F2309FF1F1B09FF1FD1
:102570002109FF1F2C09FF1F0010004010B5002982
:1025800001D001F0A5FB10BDF7B5604B0191997822
:10259000A1239B004B435E4A060014681022E418F6
:1025A000D6235B00E0583623FF33E35C00279343D8
:1025B000222B41D1574B0F3A1A600760012501F0D9
:1025C00007FD019B1880E8235B00E35C002B01D032
:1025D000B34258DD0023504FFB70AD33FF33E35857
:1025E0001A68002A03D09B88DB439B071DD0382341
:1025F000FF33E35C002B18D09B235B00E35C002BD4
:1026000013D1D133FF33E35CB3420EDAA4235B0072
:10261000E15AE018090A023101F08AFC2300012284
:10262000FE33013E01351A87FA70E8235B00E35C54
:10263000002B2AD0A8B2FEBD03683D00002BBED0FF
:1026400081880430090A023101F072FCD6235B0054
:10265000E3581F60B2E72300B133BA00FF33985844
:10266000013781880430090A023101F061FCE82356
:102670005B00E35CBB42EEDCE822F61AED180023B7
:102680005200A354A6E70027F1E7200001F070FBF9
:1026900000281FD0002E1DDD7319882647190193CD
:1026A000B600200001F0DCFC5A30800020184068A1
:1026B000013581880430090A023101F039FC20001B
:1026C00001F06EFCA3590133A351BD4202D0019B1E
:1026D0009D42E6D1114BE35C002BABD095239B00D0
:1026E000E35C002BA6D00E4BE15A0029A2D00D4A84
:1026F000A35C994202D90133A3549BE700231A211A
:102700002000A35401F074FC94E7C046300DFF1F75
:102710003409FF1F00140340E010FF1F5A0200009D
:10272000720200005E0200000D4970B54A6E0D4C49
:10273000D2038B69D20BA24206D80B4D0224AA42C7
:1027400004D901F0B5FB70BD02246442E218150003
:102750007E2425402242F4D0A3432B438B61F0E733
:1027600000F000400A200000FC1C0000F8B51D4BE2
:102770001D4F1A78002A10D1BA7B002A02D10132EB
:102780001A7003E0032AFAD0022AF8D001F0F0FB15
:1027900000220120154B1A70F8BD154B154D1C6811
:1027A000154B9E7801232B702878C0B200F0A2FB55
:1027B000BB7B002B0BD101F02BFBA1239B007343B0
:1027C000E41883239B00E41823782B70E4E7032BA1
:1027D00002D101F08DFBF0E70020022BDCD101F0EB
:1027E0008FFCEAE71C09FF1FA60BFF1F2309FF1F31
:1027F0003409FF1F490AFF1F300DFF1FF0B587B0D6
:102800000EAD2F780FAD2D780593AC4663461400BE
:102810000E4D0CAA12782E7803930D9B0092019313
:102820002200059B029701F033FB2E70012C01D092
:10283000042C08D1802206498B889343054A1278DC
:10284000D20113438B8007B0F0BDC0461C09FF1FA7
:102850006C11FF1F7809FF1F0B001B3B70B50400B4
:102860003020E02B0DD81300E025493BFF3B9BB205
:10287000ED00AB4205D8034B200019825A8201F0CB
:1028800047FA70BD8410FF1F10B501F059FA054BCF
:1028900000205B68052B04D9034A5268D20200D499
:1028A000980810BD00100040FCE100E070B501F098
:1028B000DFFB0D4B1B68FC33DC691D6AFFF7E4FF8F
:1028C0006419844204D2094B01241B68002B07D0F1
:1028D00004220024064B1A70064A9369013393615F
:1028E00001F08EFA200070BD1C65FF1F9809FF1FC4
:1028F0002309FF1FFC0FFF1F70B50C4D2B68FC3325
:102900005C6A01F0B5FBFFF7BFFF2B680025FC33C5
:102910009B6AE318834204D2054B1B68AB4200D18B
:10292000051B01F06DFA280070BDC0461C65FF1F35
:102930009809FF1FD722044B92009B5810B5002B1B
:1029400000D0984710BDC0460000FF1F10B501F031
:10295000D3F8FFF7EFFF2749274BCA6D274C1A40E2
:1029600084235B001343CB65254B1B68186A01F079
:10297000D7FA244B244A1A60244B254A1A60A02215
:10298000244B52001A60244B187801F0A1FA200061
:10299000224901F03DFB0023A3600233A360204BDA
:1029A0002049236003232048A36001F031FB10225B
:1029B0001E4BFF201A60802252031A60802292036D
:1029C0001A60802212041A6001F0DAFA012001F084
:1029D0002FFBFA20400001F05BFB582001F0B0FA19
:1029E000134801F05DFA012001F01AFB072001F005
:1029F000DFFA10BD00F0004000FEFEFF14100040A2
:102A00001C65FF1F000003400180063DBC00034021
:102A100034080000A40003404A0AFF1F71020000AE
:102A2000C3090000FFFF3F002810004000E100E064
:102A300030750000674E336888331B6883F308885D
:102A400001F04EFB644A6549136800200B40136097
:102A5000634B644A1B68934200D1A6E001F028FB57
:102A60000221614A13688B431360FFF76FFF5F4BCE
:102A70005F4C1878C0B201F0F3F80023A360023372
:102A8000A3605C4B0120236001F04AFA0323A3609A
:102A900001F02EF9040001F053F9050001F028F9C6
:102AA000554B186001F0E4F9544B1968621A531E33
:102AB000A14200D213008022D203934201D39B0291
:102AC0009B0A3268D16AC90700D471E04C491C0CDA
:102AD00009689BB24C4359432402090A641803262F
:102AE0004849FC3293680A6847489B1A474A076876
:102AF000126847499B18474A9A1833409208DB19D5
:102B00000A600360042B03D9013233400A6003607A
:102B10000E684149A619300001F0C2F83F4F3E4906
:102B20003B68C3183B603000019301F0F1FA3C4E62
:102B30003068081838493060884205D9019B013354
:102B40003B6001F0E5FA316001F07AF9354B1B7812
:102B5000002B0DD001F0F4F8334B621B19681218EA
:102B60008A4232D24919091B091A304801F050FA39
:102B70002F4E337A002B0ED001F0E2F8621BF16881
:102B80001218914224D94919091B091A294801F040
:102B90003FFA00233372284B83F3088801F048F88A
:102BA000002001F085FA01F0D3F801F081FA5CE72A
:102BB000DC0199000234641A5900641A09214B435C
:102BC0008033CB40A408E41889E7FA218900CCE7D8
:102BD0001A49DBE71C65FF1F1CF00040FFFFC1FF27
:102BE0000C0AFF1FB641210310000040490AFF1FD5
:102BF00014100040C3090000100AFF1F340AFF1F11
:102C0000380AFF1F200AFF1F280AFF1F1C0AFF1F88
:102C1000240AFF1FC4090000710200006008FF1FA2
:102C20002C0AFF1F1C09FF1FE408FF1F00100040B3
:102C3000740BFF1F3C10004000000020DC0500006A
:102C4000A022054B92009B5810B5002B01D098474D
:102C500010BD01F085F9FBE70000FF1FA122054B25
:102C600092009B5810B5002B01D0984710BD01F081
:102C700077F9FBE70000FF1FA222054B92009B584B
:102C800010B5002B01D0984710BD01F069F9FBE7A2
:102C90000000FF1FA322054B92009B5810B5002B8C
:102CA00001D0984710BD01F05BF9FBE70000FF1F62
:102CB000A422054B92009B5810B5002B01D09847D9
:102CC00010BD01F04DF9FBE70000FF1F70B501F0EA
:102CD00037F84F4B186000F0DBFF0400C30702D445
:102CE00000F0C6FF70BD00224A4B1A604A4B1878AC
:102CF0000138042829D800F075FF0320181C24008F
:102D0000200001F015F80128ECD0444C2378042B66
:102D10006ED100F0B5FF0028E4D000F0E1FF5820AC
:102D200001F00EF902232370DCE7200001F0E0F946
:102D3000E9E7200001F0C4F8E5E7200001F0A0F980
:102D4000E1E7200001F07CF9DDE701F029F805005A
:102D5000012808D1324B1B78053B012B03D82000FA
:102D6000FFF76EFFD1E72D4B1B78022B01D0052B0F
:102D700020D1022D28D12B4B9B7BAB431CD12000B3
:102D8000FFF76CFF264B18780128BED16405BCD430
:102D9000244925224B7B034205D1233A13405A4252
:102DA000534126331A000B7D9342AED9322001F0F5
:102DB0003FF8AAE7022D07D1194B1B78052B11D13B
:102DC0002000FFF759FFDDE7012D0BD1012B03D1C7
:102DD0002000FFF75FFF98E7062B03D12000FFF7E5
:102DE00067FF92E7200001F0BBF8022D8DD1C9E703
:102DF000032B04D10C4B987C00F0EAFF72E7072B01
:102E000000D06FE7094B987B00F01AFF6AE7C046D5
:102E10009C09FF1F9809FF1F9009FF1F2309FF1F2F
:102E20001C09FF1FA60BFF1FBC0BFF1FD40BFF1FAE
:102E3000FA210A4B0A4A49001A640A4A5A500A4AB5
:102E400004395A50094A08319A64094A5A50094AC1
:102E50005C315A50084ADA667047C0460000FF1FCE
:102E6000FD27FF1FF928FF1FAD28FF1FDD23FF1FD0
:102E70006D27FF1F7D1EFF1F511EFF1F10B500F0A5
:102E800099FE10BDF7B50B0CFF270122009300231C
:102E90003C001E001D009446019089B262469A4093
:102EA0001000084018413618B6B2FF2F02D1012E8B
:102EB00000D19FB2009802401A41AD18ADB2FF2C6C
:102EC00002D1012D00D19CB20133102BE6D1032099
:102ED000012E07D1012D04D1019B2401E4191C709E
:102EE0000138FEBD102EFCD10238102DF9D0023071
:102EF000F7E700008023F7B59C46264B264F019349
:102F00002649274A274D284C284B02281AD16046CB
:102F100038600868264E304080263603304308600B
:102F200001990978002909D11660224A2A60224AAB
:102F30002260E02219689143A03A1BE08021C90277
:102F40001160F2E766463E600F68194E3E408027EA
:102F5000FF023E430E600199097800290DD11760E8
:102F600001280ED1154A2A60154A2260E02219680C
:102F70009143C03A0A431A60F7BD8021890211606B
:102F8000EEE7E0210F4A02432A600F4A22601A68E6
:102F90008A43F0E74B0AFF1FE0000340D8000340DC
:102FA00090000340000003405000034040000340F5
:102FB000FFFFE3FF0280063D804508220180063DB9
:102FC000806608220080069880550822F8B51E4BBE
:102FD00080261A68002014003440324232D11A6828
:102FE0001A4F32431A6001223B68063093433B601C
:102FF00000F096FF0122164D2B681E432E603B68A1
:103000000A2613433B608027BF00124B1B683B42DC
:1030100011D1013EF6B2FF2E09D17E220E4B1C6863
:103020002B68E40B1440934323432B6005E00820F6
:1030300000F076FFE9E7002EEFD180222B686008D0
:1030400093432B60F8BDC046C4F000405CF00040E4
:1030500018F0004068F0004060F0004010B500F04B
:10306000BFFF01215820034A00F0A2FEFFF7AEFF88
:1030700010BDC046600AFF1F10B57822002103482A
:1030800000F02EFF00F0C4FD002010BD2468FF1FDB
:1030900070B5040000F0ECFF00230C200B4A010087
:1030A00059438D18515C00290DD0A14208D101234C
:1030B00000246B7000F084FF00F0A2FE200070BDC1
:1030C00001330A2BEBD11224F6E7C0462468FF1F18
:1030D00070B5040000F0CCFF002319001D000D4A5C
:1030E0001078002806D0A0420CD1557001310C3266
:1030F0000A29F5D1002B0AD100F08AFD00F080FEEC
:10310000002070BD5078461EB0411B18EEE700F05D
:1031100057FFF3E72468FF1FF7B504000C200023D6
:1031200084460E4D019267465F43E85D7E19A042DA
:1031300012D000280BD10A4B9C4662461B780833FC
:103140001370019B70707C557160B360FEBD0133DC
:103150000A2BE8D10320F9E70720F7E72468FF1FCF
:103160002068FF1F8020F8B5484BC0051B68C124AC
:103170008360474BFF251A68012313434361454B86
:10318000A4001A68444B40211A60444B1A68444B0F
:103190001A60444B1A59AA431A51C52292009E58EC
:1031A000AE433143802699509F583F49F6010F4066
:1031B0003E439E509E5880273602360A3043985030
:1031C00080201A5900020A4002431A5104341A5945
:1031D000364E3F04324080263A431A511A59360679
:1031E0001202120A32431A5108341A5980260A4030
:1031F00002431A51C32292009F58B446AF4337434B
:103200009F509F58294E0F4007439F509F5837406B
:1032100080263604374380269F509F5836063F024B
:103220003F0A37439F50C0221F59AF433A431A51B8
:103230001A591202120A1643C6221E5192009C58B5
:10324000AC4365462C439C509C5800250C402043C1
:103250009850C72080001A58154C1140C022120205
:103260000A431A50134B1B78DB08AB4201DC0020E9
:10327000F8BD2378002B06D0A368002B00D0984718
:1032800001350C34EEE71220F2E7C0461C44FF1F64
:103290001844FF1FB0F000401C68FF1FB4F000404E
:1032A0001868FF1F00E100E0FF00FFFFFFFF00FFC5
:1032B0002468FF1F2068FF1F030010B51F2809D8CE
:1032C000072200201340072404490A78A24313432D
:1032D0000B7010BD00230620F5E7C0462068FF1FD5
:1032E000054B06491B780A6805485B0702401B0B23
:1032F000134300200B6070472068FF1F1CF0004044
:10330000FFFFC1FF70B50C25FFF7EAFF0A4B1C78E1
:103310000A4BE4086543ED18002C01D1200070BD74
:103320002B78002B06D06B68002B00D09847013C0F
:103330000C3DF1E71220F2E72068FF1F1868FF1F1D
:103340001FB5002102220B0001910091052000F021
:103350007FFC02230B490A681A42FCD12023039305
:10336000039B5A1E0392002BFAD1074A1368002BC5
:10337000FCDA0B246C442000012100F0C9FD207808
:1033800004B010BD90C8004000C8004013B5040050
:103390000A4B0193019B002B01D1112016BDFFF7B1
:1033A000CFFF23000340044205D0052000F0B8FD04
:1033B000019B013BEDE71800F0E7C046FFFFFF0768
:1033C00007B500F055FE80220821D205936A0191CD
:1033D000002B01D10739916202210C4A1160019939
:1033E000481E01900029FAD1033111600531019185
:1033F0000199481E01900029FAD11160002B02D1D9
:103400008022D205936200F0FBFC07BD00C00040A3
:10341000F0B52D4C89B02378002B4FD1FEF7CEFAB2
:1034200002232A4F03903A681A42FCD120230693C4
:10343000069B5A1E0692002BFAD1254E3368002BAC
:10344000FCDA0120FFF7A2FF011E02D0112009B013
:10345000F0BD030003220190009005AD9F2000F015
:10346000F7FB0321280000F053FD02233A681A42BB
:10347000FCD120230793079B5A1E0792002BFAD1F9
:103480003368002BFCDA0120FFF780FF0028DDD134
:103490000398FEF7A7FAAA786B7811041B020B4376
:1034A00029780B4363601300113B0A49052B07D8A9
:1034B00001239340A3600B60012323700020C6E723
:1034C00080231B03F6E7C0460444FF1F90C800405A
:1034D00000C800409808FF1F1E4B30B55A68187886
:1034E0001D4B85B0D31859424B4101210093002355
:1034F00000F04EFC194B1A4A02259A6300221A6505
:1035000010325A658022C4219D65164B1648D2029E
:10351000DA6789004258154B80241A4080231B0427
:1035200013434350642341200393E40500F006FA5B
:10353000402000F003FA6562039D6B1E0393002D8B
:10354000FAD103236362FFF73BFFA562FFF760FF39
:1035500005B030BD1044FF1F95FFFEF700C80040C6
:10356000050001FF04E100E000E100E0FFFF00FFD3
:10357000F0B585B00700FEF721FA022305002D4CB7
:1035800022681A42FCD120230093009B5A1E00920D
:10359000002BFAD1284E3368002BFCDA0120FFF70C
:1035A000F5FE002803D01124200005B0F0BD234B08
:1035B0002360022322681A42FCD120230193019B3D
:1035C0005A1E0192002BFAD13368002BFCDA01203D
:1035D000FFF7DCFE0028E6D1194B1F6002232268AA
:1035E0001A42FCD120230293029B5A1E0292002B06
:1035F000FAD13368002BFCDA0120FFF7C7FE002860
:10360000D1D1104B2360022322681A42FCD120231F
:103610000393039B5A1E0392002BFAD13368002BAD
:10362000FCDA0120FFF7B2FE041EBCD12800FEF731
:10363000D9F9B9E790C8004000C800400100000671
:10364000A8C800400180000110B50020FFF790FFDE
:1036500010BD000010B5064B18705960FFF73CFF15
:1036600000211320034AFFF757FD002010BDC0467C
:103670001044FF1FD934FF1FF0B5040085B003923A
:103680000291FEF79BF9882263035B0B52051A43F4
:103690008023DB059D6A8023274F0092BA680026AD
:1036A00001901B039A420CD9F82326001B041E40EC
:1036B0001C4206D08022214B52025E6219680A43E6
:1036C0001A60002D0BD100F0D3FC02221C4B1A60B3
:1036D0008023DB055A62013A9A6200F091FB0023D5
:1036E000039A934220D1002D0AD100F0C1FC144B63
:1036F00003221D608023DB055A629D6200F080FB7F
:103700008023BA681B039A4208D9002E06D00022F3
:103710000A4B0C495A621A680A401A600198FEF76F
:1037200061F9002005B0F0BD009A0299D218127814
:10373000CA540133D4E7C0460444FF1F00C8004008
:1037400000C00040FFFFFEFFF0B587B0029103927A
:103750000400FEF733F9019000F08AFC8023022573
:103760000122234EDB0535605D629A6200F048FB62
:10377000204F3B682B42FCD120230493049B5A1E0C
:103780000492002BFAD11C4D2B68002BFCDA01208F
:10379000FFF7FCFD002802D0112007B0F0BD20008B
:1037A000039A029900F05CFB022304003A681A4273
:1037B000FCD120230593059B5A1E0592002BFAD1BC
:1037C0002B68002BFCDA0120FFF7E0FD051EE3D19A
:1037D00000F04EFC80230322DB0535605A629D62B7
:1037E00000F00EFB0198FEF7FDF8E0B2D5E7C04609
:1037F00000C0004090C8004000C80040F0B58024E0
:1038000089B00600FEF7DAF8E405A36A02250393FF
:10381000029000F02DFC0123304F3D606562A362F1
:1038200000F0EEFA2E4C23682B42FCD120230593A6
:10383000059B5A1E0592002BFAD12A4D2B68002BAE
:10384000FCDA0120FFF7A2FD002803D0112420009C
:1038500009B0F0BD244B2360022322681A42FCD138
:1038600020230693069B5A1E0692002BFAD12B6842
:10387000002BFCDA0120FFF789FD021EE6D11B4B6D
:1038800003211E60030001900090202000F0E0F969
:10389000022322681A42FCD120230793079B5A1E59
:1038A0000792002BFAD12B68002BFCDA0320FFF7DC
:1038B0006DFD041ECAD100F0DBFB80230322DB0573
:1038C0003C605A629C6200F09BFA039B002B01D182
:1038D000FFF776FD0298FEF785F8B8E700C00040D4
:1038E00090C8004000C800400100000694C8004095
:1038F00007B5000201910422000A01A9FFF724FF85
:103900000EBD000073B5050005240B4AA3005B4201
:103910009B1819686B46DE1D3000FFF7B3FA0228CA
:1039200004D133782B55013CEFD276BD052CFCD069
:103930000128FAD10230F8E7140900111F2807D82E
:10394000012380228340D20591680B439360704726
:103950003F2808D80123802220388340D2055169AE
:103960000B435361F3E75F28F1D8012380224038ED
:103970008340D205116A0B431362E8E71F2807D87A
:10398000012280218240C9058B6893438B60704778
:103990003F2808D80122802120388240C9054B6980
:1039A00093434B61F3E75F28F1D80122802140382F
:1039B0008240C9050B6A93430B62E8E71F2810D8C1
:1039C00080230200DB05153A1968012A06D8202257
:1039D0009143196019680A431A60704701228240B6
:1039E000F6E73F2811D880230200DB05353AD96875
:1039F000032A06D810229143D960D9680A43DA60B5
:103A0000EBE7012220388240F5E75F28E5D8422322
:103A10008022181A413B8340D205516A9943516272
:103A2000516A0B435362D8E710B50400012813D143
:103A3000A022184992050B685B015B0913430B60D8
:103A4000154B164A19681140154A0A431A6040225C
:103A500019680A431A6010BD0028FCD101000A2031
:103A600000F04EFA21000B2000F04AFAC0220A4B67
:103A7000920019680A4340211A601A688A431A6042
:103A8000B022044912060B685B015B0913430B600B
:103A9000E1E7C04614F000401CF000407F00FEFF4C
:103AA00080FD010072B6074A1368013313600422D7
:103AB000054B1A600023054A13608022D20553602B
:103AC000FEE7C0467808FF1FC0F00040C4F0004089
:103AD00005490B68002B05D1044A0A6004490A60B5
:103AE000044A13607047C046140AFF1F841E00007A
:103AF000380AFF1FC4F000400023034A1360034A42
:103B00001360034A1360704754F0004040F10040D6
:103B100044F10040002310B5184C8AB00093019383
:103B20002378012B27D06946012000F0D1FA002824
:103B300017D1009B12490293019B06AA0393114BD4
:103B400002A81B680493104B1B68059300F080F9D2
:103B500010220E4906A800F0ABF8002804D1FF237C
:103B6000237000200AB010BD0123094A074902A8AA
:103B7000237000F06DF90120F4E7C0462065FF1FB7
:103B800010290011082900110C2900112029001109
:103B90002465FF1F13B501246946012000F098FA3F
:103BA000034B00940193FFF7B5FF200016BDC046FC
:103BB000BB0B000010B5FFF79FFFFFF7EBFF0028DE
:103BC00002D0024B984710BDFEE7C046E1A20000BC
:103BD00002B4714649084900095649008E4402BCA6
:103BE0007047C04602B4714649084900095C490063
:103BF0008E4402BC7047C04603B471464908400079
:103C00004900095A49008E4403BC70470000000077
:103C100001B40248844601BC604700BFADAE00005D
:103C200001B40248844601BC604700BF6D0B01002F
:103C300001B40248844601BC604700BF7997000088
:103C400001B40248844601BC604700BFC1F70000D0
:103C500001B40248844601BC604700BF496D0100C1
:103C600001B40248844601BC604700BF89140100CA
:103C700001B40248844601BC604700BFDD0A010070
:103C800001B40248844601BC604700BF01D7000070
:103C900001B40248844601BC604700BFBD0B01006F
:103CA00001B40248844601BC604700BF090E000011
:103CB00001B40248844601BC604700BFCD4C0100FE
:103CC00001B40248844601BC604700BFB352010002
:103CD00001B40248844601BC604700BFE9D400003B
:103CE00001B40248844601BC604700BF6DF6000085
:103CF00001B40248844601BC604700BF156B010057
:103D000001B40248844601BC604700BF8D820000B8
:103D100001B40248844601BC604700BF116E000038
:103D200001B40248844601BC604700BF0D52010047
:103D300001B40248844601BC604700BF0134010061
:103D400001B40248844601BC604700BFC95C010061
:103D500001B40248844601BC604700BF855201009F
:103D600001B40248844601BC604700BF51B800005E
:103D700001B40248844601BC604700BF71B0000036
:103D800001B40248844601BC604700BF21440000E2
:103D900001B40248844601BC604700BFC56D010004
:103DA00001B40248844601BC604700BFDD0C01003D
:103DB00001B40248844601BC604700BF01670100AE
:103DC00001B40248844601BC604700BFF9ED000021
:103DD00001B40248844601BC604700BF4DF90000B1
:103DE00001B40248844601BC604700BF894400001A
:103DF00001B40248844601BC604700BF8B520100F9
:103E000001B40248844601BC604700BF9DA9000080
:103E100001B40248844601BC604700BFE9F60000D7
:103E200001B40248844601BC604700BFBD5C01008C
:103E300001B40248844601BC604700BF61370100FD
:103E400001B40248844601BC604700BFD54401006C
:103E500001B40248844601BC604700BFDD3F00005A
:103E600001B40248844601BC604700BF957301005D
:103E700001B40248844601BC604700BFC16601002E
:103E800001B40248844601BC604700BFE90B010051
:103E900001B40248844601BC604700BF9D6A00002F
:103EA00001B40248844601BC604700BF8D11010087
:103EB00001B40248844601BC604700BFD1AE000097
:103EC00001B40248844601BC604700BF05340100CC
:103ED00001B40248844601BC604700BFEDA5000064
:103EE00001B40248844601BC604700BFB70E000021
:103EF00001B40248844601BC604700BF75F8000069
:103F000001B40248844601BC604700BF15A20011FD
:103F100001B40248844601BC604700BF3D71010006
:103F200001B40248844601BC604700BF018900001B
:103F300001B40248844601BC604700BFC1150100BE
:103F400001B40248844601BC604700BF79120100F9
:103F500001B40248844601BC604700BFC1A500000F
:103F600001B40248844601BC604700BFE917010064
:103F700001B40248844601BC604700BFA9D80000D4
:103F800001B40248844601BC604700BFED6B0100EC
:103F900001B40248844601BC604700BFE94C0100FF
:103FA00001B40248844601BC604700BF5976010055
:103FB00001B40248844601BC604700BFF90D01000E
:103FC00001B40248844601BC604700BF21A900003B
:103FD00001B40248844601BC604700BFCD0C01001B
:103FE00001B40248844601BC604700BFED6801008F
:103FF00001B40248844601BC604700BF53B90000C9
:1040000001B40248844601BC604700BFE9270000B4
:1040100001B40248844601BC604700BF2D6C01001A
:1040200001B40248844601BC604700BFE5120100AC
:1040300001B40248844601BC604700BF6911010019
:1040400001B40248844601BC604700BFF935010055
:1040500001B40248844601BC604700BF99B5001115
:1040600001B40248844601BC604700BFD9B00000DB
:1040700001B40248844601BC604700BF75A9000036
:1040800001B40248844601BC604700BFF535010019
:1040900001B40248844601BC604700BF851201009C
:1040A00001B40248844601BC604700BF8937010063
:1040B00001B40248844601BC604700BF016C0100A6
:1040C00001B40248844601BC604700BF85C10000BE
:1040D00001B40248844601BC604700BFE1AC000067
:1040E00001B40248844601BC604700BFC9A9000072
:1040F00001B40248844601BC604700BF0934010096
:1041000001B40248844601BC604700BF19FA0000B0
:1041100001B40248844601BC604700BF090E00009C
:10412000020000003EBE00110100000050BC001162
:10413000020000003ABE0011010000006041FF1FB4
:104140000200000058BC0011010000009862FF1F2F
:104150000200000038BE0011030000000C62FF1FC7
:1041600012000000020000003EBE0011010000002D
:1041700098BC0011020000003ABE001101000000CE
:1041800095BC001102000000A2BC00110300000059
:104190004762FF1F0200000038BE0011030000004C
:1041A0005C62FF1F020000003ABE00110100000027
:1041B00094BC001102000000A0BC0011030000002C
:1041C0001D62FF1F0200000038BE00110300000046
:1041D0003E62FF1F020000003EBE00110100000011
:1041E000D8BC0011020000003ABE0011010000001E
:1041F000A942FF1F02000000EABC001101000000FC
:10420000D3BC0011020000003ABE00110100000002
:10421000A842FF1F02000000E8BC001101000000DE
:104220006462FF1F020000003ABE0011010000009E
:10423000A742FF1F02000000E6BC001101000000C1
:10424000C3BC0011020000003ABE001101000000D2
:10425000A642FF1F02000000E4BC001101000000A4
:10426000BEBC0011020000003ABE001101000000B7
:10427000A542FF1F02000000E2BC00110100000087
:10428000B9BC0011020000003ABE0011010000009C
:10429000A442FF1F02000000E0BC0011010000006A
:1042A000B4BC001102020202020200000000000081
:1042B0000D0C00009D4B0011634B00112CBD001133
:1042C00090011D0018001800FFFF070102030405FC
:1042D00006020106000000000000000000000000CF
:1042E00000000000000000000000000000000000CE
:1042F00003000000020000003EBE001101000000AB
:104300004CBD0011020000003ABE00110100000087
:104310006443FF1F0200000056BD001101000000B1
:104320009262FF1F0200000038BE0011030000006F
:10433000FC64FF1F020000003ABE001101000000F3
:104340006443FF1F0200000054BD00110100000083
:104350009462FF1F0200000038BE0011030000003D
:10436000F464FF1F126C6C6C0000000000580040E9
:10437000151600000001000000000111FFFF000001
:104380005048593600000000000000000B000500F6
:10439000F0000000B4000028002800283075A000BC
:1043A000A000A000A00000080008E001F00010003C
:1043B00010001000100010001000500050005000BD
:1043C00010001000D0070000000000000F000100E6
:1043D0000500307507001000010081FF000000009B
:1043E000FF000000FD73001105720011956F0011B0
:1043F000FFFF0100FF000000199E0011959B0011B6
:10440000AD9A00110000000000000000000008004C
:10441000040000003B0001085902E0018821280047
:10442000FF000000020000003EBE0011010000007D
:1044300004BF0011020000003ABE0011010000009C
:10444000A144FF1F0200000036BE00110100000061
:10445000DC68FF1F020000003ABE001101000000EE
:10446000A044FF1F0200000034BE00110100000044
:104470009E44FF1F020000003ABE00110100000030
:104480009C44FF1F0200000032BE0011010000002A
:104490009444FF1F180018001D0090010200000343
:1044A00002020000020000003EBE001101000000F8
:1044B00018BF0011020000003ABE00110100000008
:1044C000E444FF1F0200000030BE001100000000A5
:1044D000000000000200000038BE001103000000D0
:0644E000FC68FF1F20FF35
:040000051FFF184180
:00000001FF
